:10138200202020202025356C75204B487A200053E0
:10139200746172743A2025356C75204B4800537481
:1013A2006F703A202025356C75204B4800537465C8
:1013B200703A2020253464204B487A2000202020D7
:1013C2002025356C64204B487A20200041646A75E0
:1013D20073743A202025312E33662000204F666632
:1013E2007365743A202025336C642020002020632A
:1013F20074657374206F6666203F202020002020D1
:10140200637465737420617573203F20202000206F
:10141200206374657374206F6E203F2020202000AB
:10142200202063746573742065696E203F2020203C
:101432000044656C61793A2020253364206D732065
:1014420020002025352E3166202D6A25352E326664
:101452002020002025352E3166202B6A25352E329C
:10146200662020002020202025322E3266202020D7
:1014720020644220200020202020202025332E32EC
:10148200662020202020200020202020202020252F
:10149200342E3266202020202000202020202025EB
:1014A200332E3266202020202020200020202020E1
:1014B2006E656761746976652020202000202020F7
:1014C20020206E656761746976202020200020202C
:1014D2002020202025322E336620202020200020AC
:1014E200202020202020202020202020202020001A
:1014F20025357500242400253031662056003A2512
:10150200357520003A253566200020202020202035
:10151200200020202023203A202025326420202071
:10152200202020002020202025356C6420204B48DC
:101532007A20004572726F722025337520537765C9
:101542006570204652414D20444154412021007291
:101552003A252B30356620006A3A252B3035662035
:101562000073773A252B303566200061723A252BBD
:10157200303566200070683A252B30356620002011
:1015820041444330203A2025312E34662056002033
:1015920041444331203A2025312E34662056004101
:1015A2006E74656E6E6120416E616C797A6572202F
:1015B2002020444C354D45412056312E336B2000BE
:1015C200416E742E20416E616C797361746F72206A
:1015D200202020444C354D45412056312E336B207E
:1015E200004E6F2073657475702C207573696E6779
:1015F20020202064656661756C7420736574757053
:101602002000205374616E646172642053657475A6
:1016120070202020776972642062656E75747A7416
:1016220021200053454C2020203C2020203E202019
:101632002043520053454C202020202020202020EF
:10164200202043520053454C2020202020202020DF
:1016520020202020200020202020202020202020A8
:101662002020202043520053454C20203C3C202087
:10167200203E3E202073200020204D65617375724C
:10168200656D656E7420202000204D656173757252
:10169200652E20526573756C74002020205265748B
:1016A20075726E204C6F7373202000205265747522
:1016B200726E204C6F737320466163002020506865
:1016C20061736520466163746F7220200020205090
:1016D200686173652044656772656520200020207B
:1016E20020204D61676E697475646520202000209A
:1016F200202020496D6167205061727420202000F3
:10170200202020204672657175656E637920202045
:10171200002020202020202053575220202020204B
:101722002000202020204D657373756E67202020D5
:101732002020002020202045726765626E69732098
:101742002020200052FC636B666C2E2044E46D70F6
:1017520066756E670052FC636B666C2E2044E46D06
:1017620070662E2046002050686173656E204661C7
:101772006B746F72202000202050686173652069AD
:101782006E20477261642000202020204D61676E28
:1017920069747564652020200020496D6167696E57
:1017A200E472205465696C202000202020204672BB
:1017B200657175656E7A202020200020202020206F
:1017C2002020535752202020202020002020204378
:1017D200616C6962726174696F6E202000205368C7
:1017E2006F7274656E20496E70757420200020201F
:1017F200204F70656E20496E7075742C2020207405
:1018020068656E2068697420456E746572200043B5
:10181200616C6962722E2020204F50454E202000BC
:1018220043616C6962722E20202053484F5254202B
:101832000043616C6962722E2072656164792021B5
:1018420020002056434F2041646A7573746D656EA3
:1018520074200044656661756C74205365747570FC
:10186200203F200020204B616C69627269657275AD
:101872006E6720200045696E67616E67206B757226
:101882007A7363686C2E0045696E67616E67206FBC
:101892006666656E2020202020456E746572206485
:1018A20072FC636B656E20004B616C6962722E2064
:1018B200206F6666656E2020004B616C6962722E35
:1018C200202067657363686C2E004B616C696272DD
:1018D2002E2066657274696721200020204E6F7485
:1018E2002073686F7274656E2C202053454C202043
:1018F20020202020202020636F6E74004B65696ECB
:10190200204B75727A7363686C75737353454C2000
:101912002020202020207765697465720020202015
:10192200204E6F74206F70656E2C20202053454C22
:10193200202020202020202020636F6E7400202091
:101942004E69636874206F6666656E2C202053456D
:101952004C202020202020207765697465720020A9
:1019620056434F204B6F7272656B74757220200064
:101972005374616E646172647365747570203F2084
:101982000020202020202054657374202020202055
:1019920020002020202020204144433020202020ED
:1019A20020200020202020202041444331202020DC
:1019B20020202000202020202020536574757020D4
:1019C2002020202000202020204C616E6775616756
:1019D2006520202020002020202020537072616387
:1019E200686520202020002020202020456E676C82
:1019F2006973682020202000202020202044657563
:101A020074736368202020200020565265662041AE
:101A1200646A7573746D656E740020565265662033
:101A22004B6F7272656B7475722000204469616736
:101A32006E6F736973206F6E203F200020446961CE
:101A4200676E6F736520616E203F2020002020505A
:101A52004C4C207365742064656C617920002050C1
:101A62004C4C2F4D6573732044656C6179200020C6
:101A72002020637465737420736574757020200070
:101A820020206374657374204175737761686C20DC
:101A92000020202020205377656570202020202000
:101AA2002000202020202050726F66696C202020A8
:101AB20020200020202052756E205377656570200B
:101AC2003F20200050726F66696C207374617274DB
:101AD200656E203F002053746172742F53746F70CF
:101AE2002F537465702020206D697373696E6721AE
:101AF2002020202020002053746172742F53746FB1
:101B0200702F5374657020202020206665686C74E5
:101B120021202020202000506572666F726D696E50
:101B2200672073776565700050726F66696C20611B
:101B320075667A656963682E002020537765657043
:101B4200202072656164792020002050726F6669DE
:101B52006C2066657274696720200020525332330C
:101B620032205472616E73666572200020525332C5
:101B72003332205472616E736665722000202053E6
:101B82007765657020446174612020202000202048
:101B920050726F66696C20446174656E2020004348
:101BA200616C6962726174696F6E20446174610074
:101BB2005472616E73666572696E67204461746106
:101BC2002020746F205043202C20776169742120DB
:101BD20000204B616C696272696572646174656E42
:101BE2002000446174656E7472616E736665722062
:101BF2007A752020205043202C2077617274656E04
:101C02002021005472616E736665722020726561D4
:101C1200647920005472616E736665722066657223
:101C22007469672000202053657475702073746F87
:101C320072656420202020202020202020202020C7
:101C4200202020202000202045696E7374656C6C72
:101C5200756E67656E202020206765737065696305
:101C620068657274202000202053797374656D209A
:101C72004572726F72202000202053797374656D53
:101C82006665686C6572202000204652414D2072C4
:101C92002F77204572726F722000204652414D20EC
:0B1CA200722F77204665686C657200A9
:1060D30058767311040A111F111100110E111111B9
:1060E300110E001100111111110E0020262920207C
:1060F300202020202020202020202020202020209D
:10610300202020202020202020202020202020208C
:046113002020200028
:0300030002528521
:0D528500C0E0C0F0C083C082C0D075D0086A
:10529200908003E0FF540F640F703B9076F6E0FDC0
:1052A20090001EE475F00112074BFAC3E5F09DEA87
:1052B2009400401690001EE4F0A3F0EF9076F730D1
:1052C200E4057402F080037401F09076AE1209A036
:1052D200000003E8800312669C908002E090770A47
:0852E200F05388FDD2A8D2AF01
:0B52EA00D0D0D082D083D0F0D0E032D2
:03000B0002519D02
:0B519D00C0E0C083C082C0D075D010FD
:1051A800908003E0540FFFC2A9C28CC28D9076A1F3
:1051B800E06017EFB40F07E4F05388FD8041758A6B
:1051C80000758C7FD2A9D28C8035EF24F56013242A
:1051D800FE601714601C240770209076A17401F0FB
:1051E800801D9076A17402F080159076A17403F06A
:1051F800800D9076A17404F080059076A1E4F0D239
:01520800AFF6
:09520900D0D0D082D083D0E03275
:0300130002000EDA
:03000E00C2AF324C
:03001B0002670475
:07670400C28EC2ABD2AF321E
:030023000266B4BE
:0A66B400309904D20DC299D2AF3222
:0300730002001177
:0100110032BC
:03001600026690EF
:105A140090771FE4F0A37400F0A37439F0A374101A
:075A2400F07BFF7A167925E3
:0B5A2B0090771CEBF0A3EAF0A3E9F079
:105A3600E4FF90771CE0FBA3E0FAA3E0F98F827500
:105A46008300120683FE90771FE0FBA3E0FAA3E033
:105A5600F98F82758300EE1206C2907722E0FE0F60
:055A6600EFC39E40CDDE
:015A6B002218
:03001E008F992295
:046628007FF47E017C
:10662C00EF1F70011E144E6008907753E014F08039
:01663C00EF6E
:01663D00223A
:0B6690007D0A7F587E1B12662CDDF790
:01669B0022DC
:0C669C00E4F58AF58CD2A9D28CC28D22C4
:103B7300E4907714F07580FF7590FFF5A075B0FFA2
:103B83009076AE1209A0000003E890764F1209A0C8
:103B9300000000001266C8E4F588758921D288C246
:103BA3008AF58AF58CF5A8D2AF124AFA908002E022
:103BB300907715F0C2AFC2ABC28E12650B7BFF7A52
:103BC3001579A1125F1D120016C2AFE4907715F0AC
:103BD300FB7A0079537D20FCFFFE124C44EF700307
:103BE300023D807853E664AA6003023D7E08E664E2
:103BF300556003023D8008E690769AF008E6FFE4FC
:103C0300FCFDFE78181208C69076D21209949076BD
:103C1300D2E0F8A3E0F9A3E0FAA3E0FBC0007857F1
:103C2300E6FFE4FCFDFE78101208C6D000EB4FFF60
:103C3300EA4EFEE94DFDE84CFC9076D212099490D1
:103C430076D2E0F8A3E0F9A3E0FAA3E0FBC00078A2
:103C530058E6FFE4FCFDFE78081208C6D000EB4FDF
:103C6300FFEA4EFEE94DFDE84CFC9076D212099432
:103C73009076D2E0F8A3E0F9A3E0FAA3E0FBC0005A
:103C83007859E6FFD000EB4FFFEAFEE9FDE8FC9030
:103C930076D2120994785AE6FFE4FCFDFE781812F6
:103CA30008C6907664120994907664E0F8A3E0F96C
:103CB300A3E0FAA3E0FBC000785BE6FFE4FCFDFEB3
:103CC30078101208C6D000EB4FFFEA4EFEE94DFD17
:103CD300E84CFC907664120994907664E0F8A3E0D3
:103CE300F9A3E0FAA3E0FBC000785CE6FFE4FCFD87
:103CF300FE78081208C6D000EB4FFFEA4EFEE94DEE
:103D0300FDE84CFC907664120994907664E0F8A385
:103D1300E0F9A3E0FAA3E0FBC000785DE6FFD00082
:103D2300EB4FFFEAFEE9FDE8FC9076641209947814
:103D33005EE69076EAF008E6A3F008E6A3F008E66C
:103D4300A3F008E6900019F008E6FFE4FCFDFE7816
:103D5300081208C690763CE04EFEA3E04FFF907633
:103D63003CEEF0FAA3EFF0FB7864E6FFEAFEEB4FDC
:103D7300FF90763CEEF0A3EFF0800880009077157B
:103D83007401F0907715E0600312571712653090B5
:103D930076EAE0FCA3E0FDA3E0FEA3E0FF90769BC0
:033DA3000209947E
:105717007BFF7A1579E3125F1D120016E490769AE3
:10572700F09076D21209A000003A98907664120998
:10573700A0000186A090769B1209A03FEA233A9029
:10574700769BE0FCA3E0FDA3E0FEA3E0FF9076EAF2
:105757001209949000197407F090763C7401F07464
:105767002C124568907664E0FCA3E0FDA3E0FEA35D
:06577700E0FFA30209940B
:04456800A3F07F013C
:10456C00907719EFF0785376AA08765590769AE002
:10457C0008F69076D2E0FCA3A3A3E4FFFEFDEC7852
:10458C00181208B37856A6079076D2A3E0FDA3A321
:10459C00E4FFFEE4FC78101208B37857A607907677
:1045AC00D2A3A3E0FEA3E4FFE4FDFC78081208B359
:1045BC007858A6079076D2A3A3A3E0FF08A607908D
:1045CC007664E0FCA3A3A3E4FFFEFDEC78181208CC
:1045DC00B3785AA607907664A3E0FDA3A3E4FFFE8C
:1045EC00E4FC78101208B3785BA607907664A3A35A
:1045FC00E0FEA3E4FFE4FDFC78081208B3785CA6A7
:10460C0007907664A3A3A3E0FF08A6079076EAE0E0
:10461C0008F6A3E008F6A3E008F6A3E008F690007D
:10462C0019E008F690763CE0A308F6E008F67B006B
:10463C007A0079537D207C00E4FFFE1250B5900087
:10464C000CEFF0900018E06003020026907719E060
:10465C00604790769AE014601C04703390771FE4E6
:10466C00F0A37400F0A37429F0A37420F07BFF7AFC
:10467C001C7927801790771FE4F0A37400F0A374C3
:10468C0029F0A37420F07BFF7A1C7948125A2B1264
:0A469C005F177F307E7512662C2236
:104424009076F21209949076F2E0FCA3E0FDA3E00A
:04443400FEA3E0FF04
:0644380090771A120994AE
:10443E00209524D294D293D2929077021209A0465C
:10444E009C4200907702E0FCA3E0FDA3E0FEA3E017
:10445E00FF1203BF125F6490771AE0FCA3E0FDA386
:10446E00E0FEA3E0FF907664E0F8A3E0F9A3E0FAA3
:10447E00A3E0FBEF2BFFEE3AFEED39FDEC38FC909E
:10448E00771A120994E47B80FAF9F890771AE0FC17
:10449E00A3E0FDA3E0FEA3E0FF1208029077221234
:1044AE000994E47F80FEFDFC907722E0F8A3E0F90A
:1044BE00A3E0FAA3E0FB120777A804A905AA06ABAE
:1044CE000790771AE0FCA3E0FDA3E0FEA3E0C39BF8
:1044DE00FFEE9AFEED99FDEC98FCA31209949077ED
:1044EE0022E0FCA3E0FDA3E0FEA3E0FF78081208A3
:1044FE00C6A3120994907726E0F8A3E0F9A3E0FA98
:10450E00A3E0FBC00090771EE0FCA3E0FDA3E0FE5D
:10451E00A3E0FF78011208C6D000EB4FFFEA4EFE73
:10452E00E94DFDE84CFC907726120994907726E031
:10453E00FCA3E0FDA3E0FEA3E0FF125F6490763CD7
:10454E00E0FCA3E0FDE41203867B4D7A55795578A5
:0A455E004212016E1203BF02662C28
:10653000D294D293D2927F217E4E7D007C00125F56
:10654000649076D2E0FCA3E0FDA3E0FEA3E0FF02AE
:026550004438CD
:065F640090772A12099457
:105F6A007B1290772AA3E0FDED5404FDED6004C294
:105F7A00938002D29390772AE0FCA3E0FDA3E0FE8F
:105F8A00A3E0FF78011208C690772A120994C294F6
:105F9A00C294C294C294D294AF031BEF70C4C2924B
:085FAA00C292C292C292D2928F
:015FB20022CC
:1065730074082FFF9076E0E0146008146004147030
:0F658300031F1F1F7B007A007929AD07025C7B85
:0549A800907718EFF00C
:1049AD0014604014605224026003024A3AE4907786
:1049BD0019F090772474FFF0A37413F0A37482F0B0
:1049CD009076E1E0FCA3E0FDA3E0FEA3E0FF90778D
:1049DD00271209947B007A00792912306C78387689
:1049ED0020804A9077197402F090772474FFF0A319
:1049FD007413F0A3749180139077197402F090776B
:104A0D002474FFF0A37413F0A374A0F09076E1E08A
:104A1D00FCA3E0FDA3E0FEA3E0FF9077271209942D
:104A2D007B007A00792912306C7838767A125F170C
:104A3D00907719E0FF126573907718E07006907605
:044A4D00E112442D01
:014A51002242
:10595C0090772474FFF0A37413F0A374AFF09076D7
:10596C008CE0FFA3E0907727CFF0A3EFF07B007AD9
:10597C0000792912306C90771FE4F0A37400F0A327
:10598C007439F0A37410F07BFF7A167969125A2BD4
:10599C00125F177F099076E9E01460041470021FFF
:0C59AC001F7B007A007929AD07025C7BAC
:06670B00EF24FF92B5220D
:03671100D2B422DD
:03671400C2B422EA
:05000600C2B4D2B422D7
:103DA600E4907721F0907721E0FFC3940A5005E074
:103DB60004F080F1EF25E02423F582E43477F583DF
:103DC600E4F0A3F0EF25E02437F582E43477F583B9
:103DD600E4F0A3F0907721F0125127EF90769F60E0
:103DE60014E0FCA3E0FD907721E025E02437F5827E
:103DF600E434778012E0FCA3E0FD907721E025E033
:103E06002423F582E43477F583ECF0A3EDF0125128
:103E160027EF90769F6014E0FEA3E0FF907721E005
:103E260025E02437F582E434778012E0FEA3E0FF34
:103E3600907721E025E02423F582E43477F583EEBC
:103E4600F0A3EFF0907721E004F0E0C3940A4088F5
:103E5600E4907722F090774B1209A000000000E46E
:103E6600907721F0907721E0FFC3940A5058EF2510
:103E7600E02423F582E43477F583E0FEA3E04E6088
:103E86003D90774BE0F8A3E0F9A3E0FAA3E0FB90BE
:103E96007721E025E02423F582E43477F583E0FEFC
:103EA600A3E0FFE4FCFDEB2FFFEA3EFEED39FDEC5F
:103EB60038FC90774B120994907722E004F09077C3
:103EC60021E004F0809E907722E0FBE4FAF9F89076
:103ED600774BE0FCA3E0FDA3E0FEA3E0FF1208029F
:103EE600907632EEF0A3EFF090774F1209A0000023
:103EF6000000E4907722F0907721F0907721E0FFA0
:103F0600C3940A5058EF25E02437F582E43477F558
:103F160083E0FEA3E04E603D90774FE0F8A3E0F922
:103F2600A3E0FAA3E0FB907721E025E02437F582B1
:103F3600E43477F583E0FEA3E0FFE4FCFDEB2FFF1E
:103F4600EA3EFEED39FDEC38FC90774F120994906D
:103F56007722E004F0907721E004F0809E907722AB
:103F6600E0FBE4FAF9F890774FE0FCA3E0FDA3E06C
:0F3F7600FEA3E0FF120802907639EEF0A3EFF001
:013F85002219
:10512700E4FF12670B126711D2B3E490769FF0A3E6
:10513700F0FD0F12670B0F7E0012662C1267117FAE
:10514700027E0012662C12000612000612000612DA
:105157006714A2B3E433FC802DAF050DEFC3940CA5
:1051670050291267149076A0E025E0FF90769FE023
:1051770033FEF0A3EFF0A2B3E433FBEF4BFF9076DF
:105187009FEEF0A3EFF012671180CE126711E4FFD4
:0551970012670BAF04DC
:01519C0022F0
:104AFA00908003E0540390766EF07403F024FD7006
:104B0A000F90001374F7F0908002F0908001E4F0A7
:104B1A007FE87E0312662C1266E41266FC12665166
:104B2A001266281266511266281266511266287495
:104B3A00201266531266287F281266637F0812665F
:104B4A00637F011266637F061266637F0C126663D7
:104B5A00E4FF1266A8E4907716F0A3F0907717E0C6
:104B6A002473F582E43476F583E0FF1262F49077D9
:104B7A0017E004F07006907716E004F0C3907717F8
:104B8A00E09418907716E06480948040CF7F80127A
:054B9A0066630266BE27
:0562F400907722EFF09D
:1062F9001265921266FC907722E054F0FF908001BB
:10630900E0540F4FFEF0126657907722E0540FC405
:0F63190054F0FF908001E0540F4FFEF0026657E2
:10666300907721EFF01266E4907721E0FF0262F465
:104D7F0090771CE0FBA3E0FAA3E0F9A3E0F58275BE
:0A4D8F008300120683FF907720F0E6
:104D9900907721EFF01266EC907721E01209F14D3E
:104DA900E7B04DEFB54DF7C44DFED64E06DC4DDFED
:104DB900DF4DC7E44DCFF64DD7FC00004E0C907780
:104DC9002174E1F0803D90772174EFF08035907780
:104DD9002174F5F0802D90772174E2F08025907789
:104DE9002174DFF0801D90772174E4F08015E49040
:104DF9007721F0800E9077217401F0800690772159
:0B4E09007402F0907721E0FF0262F4D9
:0A66BE007F011266637F020266632B
:0C66A800EF33333354F82440FF026663E4
:0866E400908001E054FEF02259
:0866EC00908001E04401F0225E
:0866F400908001E04402F02255
:0866FC00908001E054FDF02242
:066651007430908001F09E
:0C665700908001E04404F0E054FBF022CD
:10615C00908001E05401FF1266E41266F490001383
:10616C007477F0908002F0908001E04404F0E054E9
:10617C0080FEE054FBF0EE5480C41313135401FE64
:10618C0090001374F7F0908002F0908001E04FF0D3
:02619C00AF064C
:01619E0022DE
:106592009077231209A000FFFFFF12615CEF600EEB
:0E65A20090772374FF120920EC4D4E4F70ECE1
:0165B00022C8
:095F14001261DF7B007A0079299B
:0B5F1D0090771CEBF0A3EAF0A3E9F082
:105F2800E4A3F01266BE7F327E0012662C7F0C124C
:105F38006663124D7F90771FE0FF04F0EFC3940F64
:105F480040F07FC0126663124D7F90771FE0FF0418
:0C5F5800F0EFC3941F40F07F0C02666362
:0E5C7B0090771AEBF0A3EAF0A3E9F0A3EDF0A6
:105C8900E4A3F07F021266637F907E0112662C7F87
:105C99000E12666390771AE0FBA3E0FAA3E0F9908D
:105CA900771EE0F582758300120683FF90771FF057
:105CB900124D9990771DE0FFA3E0FE04F0EEC39F1B
:075CC90040D27F0E0266636A
:104C4400907721ECF0A3EDF0A3EBF0A3EAF0A3E955
:014C5400F06F
:104C5500E4A3F0A3F0A3F0FD12628AEF600690775B
:104C6500287401F0907728E0606DE4F0C290D2914D
:104C75007F0112663EEF605F9077287401F09077B0
:104C850021E0FEA3E0FFC3907727E09F907726E021
:104C95009E5023E4FF1263EB907723E0FBA3E0FA39
:104CA500A3E0F9A3E475F00112076185F082F583AD
:104CB500EF1206C280C87F011263EB907723E0FBF9
:104CC500A3E0FAA3E0F9A3E475F00112076185F00A
:0F4CD50082F583EF1206C21266DB907728E0FFAC
:014CE40022AD
:0850AD007F007B017A007928E5
:1050B50090771AECF0A3EDF0A3EBF0A3EAF0A3E9E7
:0150C500F0FA
:1050C600E4907720F0A3F090771FF0FD12628AEF4C
:1050D600604690771AE0FEA3E0FFC3907721E09F39
:1050E600907720E09E503190771CE0FBA3E0FAA376
:1050F600E0F9907720E475F00112076185F082F5FA
:1051060083120683FF1262BFEF600890771F740157
:10511600F080BFE490771FF01266DB90771FE0FF08
:015126002266
:08628A00907729EEF0A3EFF07C
:10629200E4A3F0AF0512663EEF601C907729E0FFA1
:1062A2001262BFEF601190772AE0FF1262BFEF60C7
:0C62B2000690772B7401F090772BE0FF32
:0162BE0022BD
:10663E0090772CEFF01266D290772CE044A2FF12E6
:03664E0062BF2206
:0966D200D290D291C290C2912233
:0966DB00C291C290D291D290222A
:1063EB007E08E4FDD290D291ED25E0FDA290E4333E
:1063FB004DFDC291DEF0EF700AC290D291C291D2E4
:0B640B00908006D290D291C291AF05A4
:016416002263
:1062BF007E08EF30E704D2908002C290EF25E0FF16
:1062CF00D291C291DEECD290D291A290E433FFC270
:1062DF0091D29060069000187481F0EF70047F01E6
:0462EF0080027F00AA
:0162F3002288
:0A66C800D290D2911266D20266DB76
:10650B00759844758BFD758DFD758780758920C2D7
:10651B008BC2ABD28EC20BE490763BF0C298C2AC6E
:05652B00C29CC20D221C
:056552007F4112001E54
:1065570074FFFFFE209910200D0DEF1F70011E1410
:0B6567004E70F1D20D80EDC299C20D04
:016572002206
:106417007F0112456C90769AE014600B0470117B33
:10642700FF7A1C792780067BFF7A1C7948125F1D4B
:0A6437001200167FE87E0302662CB7
:101CAD00E4907716F0A3F09076A1E070030223DFA5
:101CBD0054C0907714F060030223BD5323F0907647
:101CCD00A1E04223E52254F0FE7F00900010E4F0E5
:101CDD00A304F0148EF0120A171D0210001DE92046
:101CED00001E6D30001EE24000218150002329604E
:101CFD000000002397E5238522F0120A171DA1107D
:101D0D00011DA710041DA410111DCB10121DD11003
:101D1D00131D8A10141DA410311DA710321DD710CC
:101D2D00331D8A10341DA410411DD110421DDD102C
:101D3D00431D8A10441DA410511DD710521DE310D0
:101D4D00531D8A10541DA410611DDD10621DCB1092
:101D5D00631D8A10641DA410711D8A10741DA410BA
:101D6D00811DCB10831D8A10841DA410911DE310BD
:101D7D00921DA710931D8A1094000023979076E072
:101D8D00E0FF04F0EFC394034002E4F0E4FF1249D6
:101D9D00A80222270221E9021FB69076D2E0FCA309
:101DAD00E0FDA3E0FEA3E0FF9076E11209949076AA
:101DBD004F1209A000000FA0125C24022397125BA2
:101DCD00CC022397125A6C022397125AC4022397FE
:101DDD00125B1C022397125B74022397E523852265
:101DED00F0120A171E3520011E3E20041E4A202126
:101DFD001E4D20241E3E20311E3E20411E5A2044E1
:101E0D001E6720511E4A20611E3E20621E3E206329
:101E1D001E4A20641E4A21011E4D21041E4A211115
:101E2D001E5A211400002397907643E06076021E1F
:101E3D00C29076AC7401F012564502239702236DC1
:101E4D009000147420F0A37431F0022397900014C5
:101E5D007420F0A37451F002239712535F0223975D
:101E6D00E5238522F0120A171EB130011EB430048D
:101E7D001EC230111EC830121EC830131ED63014AB
:101E8D001EB430211EB430241EC230311EB4303287
:101E9D001EB430331EDC30341EC830411EC83044F1
:101EAD0000002397021FDA74FF907706F0A3F0125B
:101EBD00638C02239712600002239774FF907706BC
:101ECD00F0A3F01263BC0223971265B1022397129F
:101EDD0065CA022397E5238522F0120A171FB64023
:101EED00011FBC40041FDA4011204E4012215A4000
:101EFD00131FE040141FBC40211FE040221FE04093
:101F0D00231FC640241FBC40311FE040321FE0405C
:101F1D00331FC640341FDA4071210E4072208840B5
:101F2D00731FD740741FDA4081208E4082204E40AF
:101F3D0083202F4084208840911FEE40921FE64061
:101F4D0093205440941FDA40A1208840A21FBC402A
:101F5D00A320E140A4204E40B1209C40B2209440EB
:101F6D00B3203540B41FDA40C1215A40C2208E4003
:101F7D00C3210040C4210E40D1210040D221004098
:101F8D00D3210640D41FDA40E11FBC40E2210E40B0
:101F9D00E3215440E4215A40F1213940F2211C4003
:101FAD00F3216B40F400002397124F2902239790E1
:101FBD00769AE0907628F0800B907628E090769ACD
:101FCD00F0126417125CD002239712571712604754
:101FDD000223971257DE022397907716E4F0A3049D
:101FED00F0907716E07002A3E090766F7018E0FC29
:101FFD00A3E0FDA3E0FEA3E0FF7B6F7A1279837867
:10200D003A1200798016E0FCA3E0FDA3E0FEA3E008
:10201D00FF7B6F7A127983783A12007D90766F127A
:10202D00099412608E022397907668E0FCA3E0FD80
:10203D00A3E0FEA3E0FF9076641209947F011245A0
:10204D006C125D7602239790766FE0FCA3E0FDA302
:10205D00E0FEA3E0FF90769B12099490769BE0FC46
:10206D00A3E0FDA3E0FEA3E0FF9076EA12099490B1
:10207D000019E054FEF07F0112456C12577D0223CA
:10208D0097125D23022397907716E4F0A304F09046
:10209D007716E07002A3E0907668601AE0FCA3E08A
:1020AD00FDA3E0FEA3E024FFFFEE34FFFEED34FFC1
:1020BD00FDEC34FF8015E0FCA3E0FDA3E0FEA3E002
:1020CD002401FFE43EFEE43DFDE43CFC9076681205
:1020DD0009948019907664E0FCA3E0FDA3E0FEA3D3
:1020ED00E0FFA3120994900019E054FDF01259B8C5
:1020FD00022397124EA0022397907631E0907643FB
:10210D00F0907643E0907631F0125DC902239790FE
:10211D00770874FFF5F0120761FEE5F064014E706B
:10212D002690770804F0A374F4F0801B907708E4F0
:10213D0075F001120761AFF0FEBE010BBFF4089000
:10214D007708E4F0A304F012619F02239790763C88
:10215D00E0FFA3E0907708CFF0A3EFF08010907729
:10216D0008E0FFA3E090763CCFF0EF124568125ED9
:10217D001C022397E4907715F0E5238522F0120ACF
:10218D001721E650012231500421E95011229350BC
:10219D0012231F501321EF501421E9502122B45066
:1021AD00222272502321F5502421E95031231F5052
:1021BD0032229350332215503421E950412272506E
:1021CD0042230650432324504421E9505121E95024
:1021DD006121E950640000239702237212543302E7
:1021ED0023979077157401F09076E0E0FF04F0EFFF
:1021FD00C394034002E4F0907715E060047F018002
:10220D00027F021249A880129076E9E0FF04F0EFF8
:10221D00C394024002E4F012595CE4900010F0A364
:10222D00F00223979076D2E0FCA3E0FDA3E0FEA39D
:10223D00E0FF9000001209949076D2E0FCA3E0FD3F
:10224D00A3E0FEA3E0FF907629120994900000E030
:10225D00FCA3E0FDA3E0FEA3E0FF9076E11209945C
:10226D00E490768BF0900000E0FCA3E0FDA3E0FE8F
:10227D00A3E0FF9076E112099412646B90768BE0E7
:10228D004401F0022397907629E0FCA3E0FDA3E042
:10229D00FEA3E0FF9076E112099412649490768B80
:1022AD00E04402F0022397900002E0FEA3E0FF90CD
:1022BD00762BE0FCA3E0C39FFFEC9EFED3EF9400D2
:1022CD00EE940450067E007F01801EAD07AC06E43F
:1022DD00120386E4FBFA79807844120277E4FBFA64
:1022ED00F9783F12007D1203BF9076D6EEF0A3EF82
:1022FD00F090768CEEF0A3EFF090768CE0FEA3E0FC
:10230D00FFEE3395E0FDFC9076E1120994126683A1
:10231D0080781248CC80731256AE806EE5238522EC
:10232D00F0120A17236D6001237760042372601188
:10233D002388601223886013237C6014237260311C
:10234D002372603423726061237760622377606348
:10235D00238D606423726081237260840000239753
:10236D001252F580251255078020125E6F801B904A
:10237D0000147460F0A37421F0800F125EC2800A05
:10238D009000147460F0A37471F09076A1E0448015
:10239D00F0900010E07002A3E06037900014E0FEB2
:1023AD00A3E0FF900010EEF0A3EFF08E22F52322B4
:1023BD009076A1E054C0FFBF8018908003E0540FC9
:1023CD00907714F0E0B40F0A12669C9076A1E04469
:0223DD0040F0CE
:0123DF0022DB
:104F29009000147410F0A37401F090769AE0146064
:104F39001C04703390771FE4F0A37400F0A3742964
:104F4900F0A37410F07BFF7A16797A801790771F97
:104F5900E4F0A37400F0A37429F0A37410F07BFFAC
:104F69007A177924125A2B90771FE4F0A37400F072
:104F7900A37439F0A37410F07BFF7A167936125AAC
:104F89002B900019E0FF30E204783E7663EF30E1C0
:104F99000478417676EF30E004784476727B007AC3
:064FA900007929025F1DE2
:105C24009000147410F0A304F0E490764EF0907693
:105C34009AE014601C04703390771FE4F0A374009E
:105C4400F0A37429F0A37410F07BFF7A16798B808B
:105C54001790771FE4F0A37400F0A37429F0A374E1
:105C640010F07BFF7A177935125A2B1265FA7B00F4
:075C74007A007929025F1D8F
:105A6C009000147410F0A37431F0E490764EF09022
:105A7C00769AE014601C04703390771FE4F0A374E2
:105A8C0000F0A37429F0A37410F07BFF7A16799CB4
:105A9C00801790771FE4F0A37400F0A37429F0A38F
:105AAC007410F07BFF7A177946125A2B1265FA7B29
:085ABC00007A007929025F1D48
:105AC4009000147410F0A37441F0E490764EF090BA
:105AD400769AE014601C04703390771FE4F0A3748A
:105AE40000F0A37429F0A37410F07BFF7A1679AD4B
:105AF400801790771FE4F0A37400F0A37429F0A337
:105B04007410F07BFF7A177957125A2B1265FA7BBF
:085B1400007A007929025F1DEF
:105B1C009000147410F0A37451F0E490764EF09051
:105B2C00769AE014601C04703390771FE4F0A37431
:105B3C0000F0A37429F0A37410F07BFF7A1679BEE1
:105B4C00801790771FE4F0A37400F0A37429F0A3DE
:105B5C007410F07BFF7A177968125A2B1265FA7B56
:085B6C00007A007929025F1D97
:105B74009000147410F0A37461F0E490764EF090E9
:105B8400769AE014601C04703390771FE4F0A374D9
:105B940000F0A37429F0A37410F07BFF7A1679CF78
:105BA400801790771FE4F0A37400F0A37429F0A386
:105BB4007410F07BFF7A177979125A2B1265FA7BED
:085BC400007A007929025F1D3F
:105BCC009000147410F0A37491F0E490764EF09061
:105BDC00769AE014601C04703390771FE4F0A37481
:105BEC0000F0A37429F0A37410F07BFF7A177913DB
:105BFC00801790771FE4F0A37400F0A37429F0A32E
:105C0C007410F07BFF7A1779BD125A2B1265FA7B50
:085C1C00007A007929025F1DE6
:1052F5009000147420F0A37401F090769AE0146085
:105305001C04703390771FE4F0A37400F0A3742994
:10531500F0A37410F07BFF7A1779CE801790771F72
:10532500E4F0A37400F0A37429F0A37410F07BFFDC
:105335007A187966125A2B90771FE4F0A37400F05F
:10534500A37439F0A37410F07BFF7A167936125ADC
:0A5355002B7B007A007929025F1D0E
:105645009000147420F0A304F090769AE014601C86
:1056550004703390771FE4F0A37400F0A37429F06D
:10566500A37410F07BFF7A1779DF801790771FE41A
:10567500F0A37400F0A37429F0A37410F07BFF7AF3
:10568500187977125A2B90771FE4F0A37400F0A3D2
:105695007439F0A37410F07BFF7A167936125A2B01
:0956A5007B007A007929025F1DE7
:10535F009000147420F0A37441F090769AE01460DA
:10536F001C04703390771FE4F0A37400F0A374292A
:10537F00F0A37410F07BFF7A1779F0801790771FE6
:10538F00E4F0A37400F0A37429F0A37410F07BFF72
:10539F007A187989125A2B90771FE4F0A37400F0D2
:1053AF00A37439F0A37410F07BFF7A167936125A72
:0A53BF002B7B007A007929025F1DA4
:1053C9009000147420F0A37461F090769AE0146050
:1053D9001C04703390771FE4F0A37400F0A37429C0
:1053E900F0A37410F07BFF7A187933801790771F38
:1053F900E4F0A37400F0A37429F0A37410F07BFF08
:105409007A1879CC125A2B90771FE4F0A37400F024
:10541900A37439F0A37410F07BFF7A167936125A07
:0A5429002B7B007A007929025F1D39
:104FAF009000147420F0A37451F090769AE014607E
:104FBF001C04703390771FE4F0A37400F0A37429DE
:104FCF00F0A37410F07BFF7A187911801790771F78
:104FDF00E4F0A37400F0A37429F0A37410F07BFF26
:104FEF007A1879AA125A2B90772474FFF0A37413AE
:104FFF00F0A374BFF09076F2E0FCA3E0FDA3E0FE17
:10500F00A3E0FF9077271209947B007A0079391279
:0F501F00306C784876207B007A007929025F1D7B
:10502E009000147420F0A37431F090769AE014601E
:10503E001C04703390771FE4F0A37400F0A374295E
:10504E00F0A37410F07BFF7A187922801790771FE7
:10505E00E4F0A37400F0A37429F0A37410F07BFFA6
:10506E007A1879BB125A2B90772474FFF0A374131D
:10507E00F0A374BFF09076F2E0FCA3E0FDA3E0FE97
:10508E00A3E0FF9077271209947B007A00793912FA
:0F509E00306C784876207B007A007929025F1DFC
:10589E009000147421F0A37401F090769AE01460D5
:1058AE001C04703390771FE4F0A37400F0A37429E6
:1058BE00F0A37420F07BFF7A1879DD801790771FA4
:1058CE00E4F0A37400F0A37429F0A37420F07BFF1E
:1058DE007A1879FE125A2B125F17900014E0FEA36D
:0F58EE00E0FF900010EEF0A3EFF08E22F52322E2
:1058FD009000147421F0A37411F090769AE0146066
:10590D001C04703390771FE4F0A37400F0A3742986
:10591D00F0A37420F07BFF7A19791F801790771F01
:10592D00E4F0A37400F0A37429F0A37420F07BFFBE
:10593D007A197940125A2B125F17900014E0FEA3CA
:0F594D00E0FF900010EEF0A3EFF08E22F5232282
:106000009000147430F0A37401F090771F14F0A383
:106010007400F0A37429F0A37410F07BFF7A19794F
:1060200083125A2B90771FE4F0A37400F0A3743905
:10603000F0A37410F07BFF7A167936125A2B7B008E
:076040007A007929025F1DBF
:10638C009000147430F0A37411F090771FE4F0A314
:10639C007400F0A37429F0A37410F07BFF7A1979C0
:1063AC0094125A2B125A147B007A007929025F1D21
:1065B1009000147430F0A37421F01265E3125A14A0
:0965C1007B007A007929025F1DBC
:1063BC009000147430F0A304F090771FE4F0A374F1
:1063CC0000F0A37429F0A37410F07BFF7A1979A55F
:0F63DC00125A2B125A147B007A007929025F1D86
:1065CA009000147430F0A37441F01265E3125A1467
:0965DA007B007A007929025F1DA3
:106047009000147440F0A37401F090771F14F0A32C
:106057007400F0A37429F0A37410F07BFF7A197908
:10606700B6125A2B90771FE4F0A37400F0A374398B
:10607700F0A37410F07BFF7A167936125A2B7B0047
:076087007A007929025F1D78
:105CD0009000147440F0A37411F090769AE0146070
:105CE0001C04703390771FE4F0A37400F0A37429B0
:105CF000F0A37410F07BFF7A1979C7801790771F93
:105D0000E4F0A37400F0A37429F0A37410F07BFFF7
:105D10007A1979D8125A2B125A147B007A007929F1
:035D2000025F1D02
:1057DE009000147440F0A37421F0907628E004F049
:1057EE00D394014002E4F0907628E014601C04701B
:1057FE003390771FE4F0A37400F0A37429F0A37420
:10580E0010F07BFF7A1979E9801790771FE4F0A3E7
:10581E007400F0A37429F0A37410F07BFF7A197949
:10582E00FA125A2B125A147B007A007929025F1D44
:105D23009000147440F0A37471F090769AE01460BC
:105D33001C04703390771FE4F0A37400F0A374295C
:105D4300F0A37410F07BFF7A187955801790771FB2
:105D5300E4F0A37400F0A37429F0A37410F07BFFA4
:105D63007A197972125A2B125A147B007A00792904
:035D7300025F1DAF
:10577D009000147440F0A37481F090769AE0146058
:10578D001C04703390771FE4F0A37400F0A3742908
:10579D00F0A37410F07BFF7A1A790B801790771FA6
:1057AD00E4F0A37400F0A37429F0A37410F07BFF50
:1057BD007A1A791C125A2B125A14125F1790769B73
:1057CD00E0FCA3E0FDA3E0FEA3E0FF90766F0209ED
:0157DD009437
:10608E009000147440F0A37491F090772474FFF094
:10609E00A37413F0A374CEF090766FE0FCA3E0FD32
:1060AE00A3E0FEA3E0FF9077271209947B007A000D
:1060BE00792912306C125A14783876567B007A0091
:0560CE007929025F1DAD
:105D76009000147440F0A374A1F090769AE0146039
:105D86001C04703390771FE4F0A37400F0A3742909
:105D9600F0A37410F07BFF7A187944801790771F70
:105DA600E4F0A37400F0A37429F0A37410F07BFF51
:105DB6007A197961125A2B125A147B007A007929C2
:035DC600025F1D5C
:1059B8009000147440F0A374B1F090772474FFF051
:1059C800A37413F0A374DEF0907664E0F8A3E0F912
:1059D800A3E0FAA3E0FBA3E0FCA3E0FDA3E0FEA3A1
:1059E800E0C39BFFEE9AFEED99FDEC98FC907727BB
:1059F8001209947B007A00792912306C125A1478B3
:0C5A08003876207B007A007929025F1DAF
:105DC9009000147440F0A374C1F090769AE01460C6
:105DD9001C04703390771FE4F0A37400F0A37429B6
:105DE900F0A37410F07BFF7A1A7971801790771FEE
:105DF900E4F0A37400F0A37429F0A37410F07BFFFE
:105E09007A1A7982125A2B125A147B007A0079294C
:035E1900025F1D08
:104EA0009000147440F0A374D1F0907631E0603734
:104EB00090769AE014601204702690772474FFF0C4
:104EC000A37413F0A374EF800D90772474FFF0A304
:104ED0007414F0A37400F07B007A00792912306C0E
:104EE000E4907631F0803690769AE0146012047087
:104EF0002690772474FFF0A37414F0A37411800D2E
:104F000090772474FFF0A37414F0A37422F07B0054
:104F10007A00792912306C9076317401F0125A14AB
:094F20007B007A007929025F1D73
:105E1C009000147440F0A374E1F090769AE0146052
:105E2C001C04703390771FE4F0A37400F0A3742962
:105E3C00F0A37410F07BFF7A1A794F801790771FBC
:105E4C00E4F0A37400F0A37429F0A37410F07BFFAA
:105E5C007A1A7960125A2B125A147B007A0079291B
:035E6C00025F1DB5
:10619F009000147440F0A374F1F090772474FFF022
:1061AF00A37414F0A37433F0907708E0FFA3E0908A
:1061BF007727CFF0A3EFF07B007A00792912306CAC
:1061CF00125A14783876207B007A007929025F1DE5
:105433009000147450F0A37401F090769AE0146015
:105443001C04703390771FE4F0A37400F0A3742955
:10545300F0A37410F07BFF7A1A7993801790771F6B
:10546300E4F0A37400F0A37429F0A37410F07BFF9D
:105473007A1A79A4125A2B90771FE4F0A37400F0E0
:10548300A37439F0A37410F07BFF7A167936125A9D
:0A5493002B7B007A007929025F1DCF
:10646B009000147450F0A37411F090771FE4F0A314
:10647B007400F0A37439F0A37410F07BFF7A1679D3
:09648B0069125A2B7F010249A895
:106494009000147450F0A37421F090771FE4F0A3DB
:1064A4007400F0A37439F0A37410F07BFF7A1679AA
:0964B40069125A2B7F020249A86B
:0D6683009000147450F0A37431F002595CC3
:1048CC0090768BE064037072A3E07002A3E0606AE0
:1048DC009000147450F0A37441F090769AE0146038
:1048EC001C04703390771FE4F0A37400F0A37429B8
:1048FC00F0A37410F07BFF7A1A79B5801790771FAC
:10490C00E4F0A37400F0A37429F0A37410F07BFFFF
:10491C007A1A79C6125A2B90771FE4F0A37400F020
:10492C00A37439F0A37410F07BFF7A167936125AFF
:10493C002B7B007A007929025F1D90769AE0146037
:10494C001C04703390771FE4F0A37400F0A3742957
:10495C00F0A37420F07BFF7A1A79D7801790771F19
:10496C00E4F0A37400F0A37429F0A37420F07BFF8F
:10497C007A1A79F8125A2B125F171266909000145B
:10498C00E0FEA3E08EF0120A1749A1501149A45081
:0C499C0031000049A702646B1266832200
:1056AE009000147450F0A304F090769AE014601CED
:1056BE0004703390771FE4F0A37400F0A37429F004
:1056CE00A37410F07BFF7A1B7919801790771FE473
:1056DE00F0A37400F0A37429F0A37410F07BFF7A8A
:1056EE001B792A125A2B90771FE4F0A37400F0A3B3
:1056FE007439F0A37410F07BFF7A167936125A2B98
:09570E007B007A007929025F1D7D
:10549D009000147450F0A37461F090769AE014604B
:1054AD001C04703390771FE4F0A37400F0A37429EB
:1054BD00F0A37410F07BFF7A1B793B801790771F58
:1054CD00E4F0A37400F0A37429F0A37410F07BFF33
:1054DD007A1B794C125A2B90771FE4F0A37400F0CD
:1054ED00A37439F0A37410F07BFF7A167936125A33
:0A54FD002B7B007A007929025F1D65
:105507009000147460F0A37401F090769AE0146030
:105517001C04703390771FE4F0A37400F0A3742980
:10552700F0A37410F07BFF7A1B795D801790771FCB
:10553700E4F0A37400F0A37429F0A37410F07BFFC8
:105547007A1B796E125A2B90771FE4F0A37400F040
:10555700A37439F0A37410F07BFF7A167936125AC8
:0A5567002B7B007A007929025F1DFA
:105E6F009000147460F0A37411F090769AE01460AF
:105E7F001C04703390771FE4F0A37400F0A374290F
:105E8F00F0A37410F07BFF7A1B797F801790771F38
:105E9F00E4F0A37400F0A37429F0A37410F07BFF57
:105EAF007A1B7990125A2B125A147B007A00792997
:035EBF00025F1D62
:105571009000147460F0A37481F090769AE0146046
:105581001C04703390771FE4F0A37400F0A3742916
:10559100F0A37410F07BFF7A1C7905801790771FB8
:1055A100E4F0A37400F0A37429F0A37410F07BFF5E
:1055B1007A1C7916125A2B90771FE4F0A37400F02D
:1055C100A37439F0A37410F07BFF7A167936125A5E
:0A55D1002B7B007A007929025F1D90
:105EC2009000147460F0A304F090769AE014601CC1
:105ED20004703390771FE4F0A37400F0A37429F0E8
:105EE200A37410F07BFF7A1B79A1801790771FE4CF
:105EF200F0A37400F0A37429F0A37410F07BFF7A6E
:105F02001B79D3125A2B125A147B007A0079290278
:025F12005F1D11
:1055DB009000147460F0A37481F090769AE01460DC
:1055EB001C04703390771FE4F0A37400F0A37429AC
:1055FB00F0A37410F07BFF7A1C7905801790771F4E
:10560B00E4F0A37400F0A37429F0A37410F07BFFF3
:10561B007A1C7916125A2B90771FE4F0A37400F0C2
:10562B00A37439F0A37410F07BFF7A167936125AF3
:0A563B002B7B007A007929025F1D25
:1061DF00E4FFFE7D707C419076DCE0F8A3E0F9A34C
:1061EF00E0FAA3E0FB12031460025018E4FFFEFD77
:1061FF00FC9076DCE0F8A3E0F9A3E0FAA3E0FB1251
:0E620F00031450057839763F22783976202224
:104B9F00300903024C43C2AF9077147401F0E4FF65
:104BAF00FEFDFC907635E0F8A3E0F9A3E0FAA3E070
:104BBF00FB1203145024907635E0FCA3E0FDA3E034
:104BCF00FEA3E0FFE4FBFA798078BF12016E9076C6
:104BDF0035120994907714E014F0907714E09077E1
:104BEF0024600C74FFF0A37414F0A37444800A744F
:104BFF00FFF0A37414F0A37455F0907644E0FCA377
:104C0F00E0FDA3E0FEA3E0FF9077271209949076D2
:104C1F0035E0FCA3E0FDA3E0FEA3E0FF90772B12AD
:104C2F0009947B007A00793912306CD2AF783F76D5
:044C3F00F4125F14F8
:014C4300224E
:1063280020092E90772474FFF0A37414F0A37466E8
:10633800F0900020E0FCA3E0FDA3E0FEA3E0FF90C6
:1063480077271209947B007A00793912306C125F32
:0263580014220D
:10635A0020092E90772474FFF0A37414F0A37478A4
:10636A00F0907702E0FCA3E0FDA3E0FEA3E0FF903B
:10637A0077271209947B007A00793912306C125F00
:02638A001422DB
:10621D0090772474FFF0A37414F0A3748AF0907631
:10622D002DE0FCA3E0FDA3E0FEA3E0FF9077271295
:10623D0009947B007A00793912306C1261DF7B0092
:07624D007A007929025F1DB0
:1062540020093290772474FFF0A37414F0A3749C83
:10626400F0900024E0FCA3E0FDA3E0FEA3E0FF9097
:1062740077271209947B007A00793912306C7844BC
:0662840076B0125F142247
:1052120020096FE4FFFEFDFC9076DCE0F8A3E0F9E4
:10522200A3E0FAA3E0FB120314502990769AE0144B
:10523200601204704A90772474FFF0A37414F0A3F0
:1052420074AE800D90772474FFF0A37414F0A374ED
:10525200BFF0802290772474FFF0A37414F0A3743B
:10526200D0F09076DCE0FCA3E0FDA3E0FEA3E0FF3B
:105272009077271209947B007A00793912306C12E8
:035282005F142294
:1065E30090772474FFF0A37414F0A374E1F07B009C
:0765F3007A00792902306CE7
:1065FA0090772474FFF0A37414F0A374E1F07B0085
:07660A007A00793902306CBF
:106673001265577F0A12001E1265577F0D02001E16
:10661100C299C20D7F2412001E12655712655212D3
:0766210065527F3D02001EDF
:1064BD00907654E0FF1264DAA3E0FF1264DAA3E0F1
:0D64CD00FF1264DAA3E0FF1264DAA3E0FF1F
:0A64DA00AD07126557AF0502001E62
:1038BB009076D2E0FCA3E0FDA3E0FEA3E0FF9077BF
:1038CB0015120994900014E0FEA3E08EF0120A1773
:1038DB0038E720313A16205100003B4EE490000DA2
:1038EB00F0A3F09076D2E0FCA3E0FDA3E0FEA3E012
:1038FB00FF9077151209949076F21209A00000053B
:10390B00DC12442A123DA69077147401F09076AC29
:10391B00E0604C120A44E4FFFE7D407C409076440C
:10392B00E0F8A3E0F9A3E0FAA3E0FB1203146002B2
:10393B00501AE4FFFE7D407CC0907644E0F8A3E093
:10394B00F9A3E0FAA3E0FB1203145005E4907714FB
:10395B00F0907714E0700812589EE49076ACF090DB
:10396B007714E07003023B4E12502E12442A123D84
:10397B00A6907632E0FF90000DE0FCA3E0FD24283A
:10398B00F58274003CF583EFF0907633E0FF7429F9
:10399B002DF58274003CF583EFF0907639E0FF74DF
:1039AB002A2DF58274003CF583EFF090763AE0FF18
:1039BB00742B2DF58274003CF583EFF090000EE034
:1039CB002408F090000DE03400F09076F2E0FCA3B8
:1039DB00E0FDA3E0FEA3E02432FFE43EFEE43DFD68
:1039EB00E43CFC9076F2120994E47BEA7A88F9F8CD
:1039FB00D31208A2400302397312535F752220754C
:103A0B0023419076AC7401F0023B4EE490000DF034
:103A1B00A3F09076F21209A0000005DC12442A12E2
:103A2B003DA69077147401F09076ACE06058E4906A
:103A3B007714F0120A44E4FFFE7D7A7C43907644BF
:103A4B00E0F8A3E0F9A3E0FAA3E0FB120314600291
:103A5B00501AE4FFFE7D7A7CC3907644E0F8A3E035
:103A6B00F9A3E0FAA3E0FB12031450069077147449
:103A7B0001F0907714E0700E9076ACE0600812586D
:103A8B00FDE49076ACF0907714E07003023B4E129D
:103A9B004FAF12442A123DA6907632E0FF90000DF4
:103AAB00E0FCA3E0FD242CF58274003CF583EFF0E1
:103ABB00907633E0FF742D2DF58274003CF583EF87
:103ACB00F0907639E0FF742E2DF58274003CF5836F
:103ADB00EFF090763AE0FF742F2DF58274003CF5F1
:103AEB0083EFF090000EE02408F090000DE034001E
:103AFB00F09076F2E0FCA3E0FDA3E0FEA3E024321D
:103B0B00FFE43EFEE43DFDE43CFC9076F2120994AA
:103B1B00E47BEA7A88F9F8D31208A24003023A9AB6
:103B2B007E017DF07C141250AD90000CEFF09000F4
:103B3B0019E054FBF0E4FF12456C1253C9752220B7
:103B4B00752361907715E0FCA3E0FDA3E0FEA3E0F5
:103B5B00FF9076D21209949076D2E0FCA3E0FDA3FD
:083B6B00E0FEA3E0FF02443874
:103F86009077167401F0A3E4F09077147405F0A30B
:103F960074DCF090769AE014601C04703390771FFE
:103FA600E4F0A37400F0A37429F0A37420F07BFF5F
:103FB6007A1B79B2801790771FE4F0A37400F0A300
:103FC6007429F0A37420F07BFF7A1B79E4125A2B34
:103FD600125F17E4907718F0A3F012661190771825
:103FE600E0FEA3E07803C333CE33CED8F9FF907753
:103FF60017E02FFF907716E03EFE7B007A0079539C
:104006007D087C00124C4490000CEFF090772474ED
:10401600FFF0A37414F0A374F2F0907718E0FEA3F7
:10402600E0FF7C007D321206E4907715E02FFF90CA
:104036007714E03E907727F0A3EFF07B017A76794C
:104046005412306C1264BD7F201264DA7F4D126404
:10405600DA7F481264DA7F7A1264DA7F201264DA31
:104066007853E67F00FE90771AF0A3EFF008E6FD9E
:10407600EDFF90771AEEF0A3EFF07F201264DA7F5F
:104086004D12583E7855E67F00FE90771AF0A3EF62
:10409600F008E6FDEDFF90771AEEF0A3EFF07F5003
:1040A60012583E7857E67F00FE90771AF0A3EFF09D
:1040B60008E6FDEDFF90771AEEF0A3EFF07F4D12C4
:1040C60064DA7F4F1258437859E67F00FE90771ADC
:1040D600F0A3EFF008E6FDEDFF90771AEEF0A3EF00
:1040E600F07F501264DA7F4F1258431266731265DE
:1040F60057907719E004F07006907718E004F0C343
:10410600907719E0949F907718E094025003023F4D
:10411600E090772474FFF0A37414F0A374F6F07B98
:10412600017A76795412306C7F021264410266730A
:10583E001264DA7F431264DA7F201264DA90771AE8
:05584E00E0FEA3E0FFF5
:1058530090772474FFF0A37414F0A374F9F0AD07E8
:10586300AC06E412038690769BE0F8A3E0F9A3E08C
:10587300FAA3E0FB12016EE4FBFA79807845120289
:10588300779077271209947B017A76795412306CDA
:0B5893001264BD1264CB7F200264DAB7
:0E0A44009076F2E0FCA3E0FDA3E0FEA3E0FF4D
:060A5200907719120994CF
:100A5800907643E0602E12667390772474FFF0A3BB
:100A68007415F0A37400F090771BE0FFA3E0907773
:100A780027CFF0A3EFF07B017A76795412306C7FA0
:100A880007126441E47B32FAF9F8907719E0FCA385
:100A9800E0FDA3E0FEA3E0FF120802E47B32FAF9CE
:100AA800F812077790771DEEF0A3EFF02432FFE4F9
:100AB8003EA3F0A3EFF0907643E06056907724745D
:100AC800FFF0A37415F0A37400F090771DE0FFA366
:100AD800E0907727CFF0A3EFF07B017A7679541274
:100AE800306C7F0712644190772474FFF0A374156B
:100AF800F0A37400F090771FE0FFA3E0907727CF72
:100B0800F0A3EFF07B017A76795412306C7F0712EC
:100B1800644190771EE02424FF90771DE034FAFEAC
:100B28007C007D321206F6EF7803C333CE33CED87D
:100B3800F92400FFEE3401FEE49076E6F0FB7A003B
:100B480079537D10FC124C4490000CEFF07853E67A
:100B58007F007851F6FE08EFF67854126118907607
:100B6800C7120994907643E0603090772474FFF0C0
:100B7800A37415F0A37406F09076C7E0FCA3E0FD1B
:100B8800A3E0FEA3E0FF9077271209947B017A7611
:100B9800795412306C7F071264417857E67F0078E9
:100BA80051F6FE08EFF678581261189076F9120996
:100BB80094907643E0603090772474FFF0A3741526
:100BC800F0A37406F09076F9E0FCA3E0FDA3E0FE44
:100BD800A3E0FF9077271209947B017A7679541263
:100BE800306C7F071264417859E67F007851F6FE31
:100BF80008EFF6785A1261189076A2120994907646
:100C080043E0603090772474FFF0A37415F0A37468
:100C180006F09076A2E0FCA3E0FDA3E0FEA3E0FFCF
:100C28009077271209947B017A76795412306C7F79
:100C380007126441785BE67F007851F6FE08EFF60C
:100C4800785C1261189076A8120994907643E06057
:100C58003090772474FFF0A37415F0A37406F09015
:100C680076A8E0FCA3E0FDA3E0FEA3E0FF907727D1
:100C78001209947B017A76795412306C7F071264DA
:100C880041785FE67F007851F6FE08EFF67860124B
:100C980061189076EE120994907643E06030907770
:100CA8002474FFF0A37415F0A37406F09076EEE0B8
:100CB800FCA3E0FDA3E0FEA3E0FF907727120994D0
:100CC8007B017A76795412306C7F0712644178611F
:100CD800E67F007851F6FE08EFF678621261189008
:100CE8007692120994907643E0606390772474FFBB
:100CF800F0A37415F0A37406F0907692E0FCA3E0DC
:100D0800FDA3E0FEA3E0FF9077271209947B017A08
:100D180076795412306C7F071264411266739077AB
:100D28002474FFF0A37415F0A3740CF0907692E08D
:100D3800FCA3E0FDA3E0FEA3E0FF9077271209944F
:100D48007B017A76795412306C7F07126441907770
:100D580001E060419076C7E0FCA3E0FDA3E0FEA3BC
:100D6800E0FF90768E1209949076F9E0FCA3E0FDFE
:100D7800A3E0FEA3E0FF9076C31209949076A2E068
:100D8800FCA3E0FDA3E0FEA3E0FF9076CC1209945B
:100D9800E4907701F090771DE0FEA3E0FBAA0690AF
:100DA8007719E0FCA3E0FDA3E0FEA3E0C39BFFEE00
:100DB8009AFEED9400FDEC9400FCE4120381C0045B
:100DC800C005C006C00790771DE0FEA3E0FFC390F2
:100DD8007720E09FFD90771FE09EFCE4120386A831
:100DE80004A905AA06AB07D007D006D005D004127F
:100DF80002777825120988907643E0602790772457
:100E080074FFF0A37415F0A37406F078251208D9BE
:100E18009077271209947B017A76795412306C7F87
:100E2800071264419076C7E0F8A3E0F9A3E0FAA3BB
:100E3800E0FB9076A8E0FCA3E0FDA3E0FEA3E0FFC2
:100E480012007978251208F512016E9076C7E0F83D
:100E5800A3E0F9A3E0FAA3E0FB12007D9076A812C4
:100E68000994907643E0603090772474FFF0A3747F
:100E780015F0A37406F09076A8E0FCA3E0FDA3E0CB
:100E8800FEA3E0FF9077271209947B017A767954C4
:100E980012306C7F071264419076F9E0F8A3E0F90C
:100EA800A3E0FAA3E0FB9076EEE0FCA3E0FDA3E06C
:100EB800FEA3E0FF12007978251208F512016E9062
:100EC80076F9E0F8A3E0F9A3E0FAA3E0FB12007DCD
:100ED8009076EE120994907643E06030907724740F
:100EE800FFF0A37415F0A37406F09076EEE0FCA36F
:100EF800E0FDA3E0FEA3E0FF9077271209947B01B1
:100F08007A76795412306C7F071264419076A2E0A9
:100F1800F8A3E0F9A3E0FAA3E0FB907692E0FCA343
:100F2800E0FDA3E0FEA3E0FF12007978251208F5A2
:100F380012016E9076A2E0F8A3E0F9A3E0FAA3E02C
:100F4800FB12007D907692120994907643E060300F
:100F580090772474FFF0A37415F0A37406F09076CC
:100F680092E0FCA3E0FDA3E0FEA3E0FF9077271248
:100F780009947B017A76795412306C7F07126441A8
:100F8800123DA6907632E0FCA3E0FD1261289000A5
:100F98001A120994907643E0603090772474FFF039
:100FA800A37415F0A37406F090001AE0FCA3E0FD0A
:100FB800A3E0FEA3E0FF9077271209947B017A76DD
:100FC800795412306C7F07126441907639E0FCA3A3
:100FD800E0FD1261289076FD120994907643E06056
:100FE8003090772474FFF0A37415F0A37406F09082
:100FF80076FDE0FCA3E0FDA3E0FEA3E0FF907727E9
:101008001209947B017A76795412306C7F07126446
:10101800419076A8E0FCA3E0FDA3E0FEA3E0FF90EA
:1010280076EEE0F8A3E0F9A3E0FAA3E0FB12007D76
:10103800E4FBFAF9784012027790000412099490C0
:10104800001AE0F8A3E0F9A3E0FAA3E0FB9000049B
:10105800E0FCA3E0FDA3E0FEA3E0FF120079907698
:101068003E12099490762D1209A03BA3D70A9076D8
:10107800FDE0F8A3E0F9A3E0FAA3E0FB907692E0A4
:10108800FCA3E0FDA3E0FEA3E0FF120079900008B6
:1010980012099490762DE0F8A3E0F9A3E0FAA3E012
:1010A800FB900008E0FCA3E0FDA3E0FEA3E0FF1234
:1010B80002779000241209947B8F7AC279F5783CE4
:1010C80090763EE0FCA3E0FDA3E0FEA3E0FF120261
:1010D80077900020120994E4FBFA79A078419000F7
:1010E80020E0FCA3E0FDA3E0FEA3E0FF120277905E
:1010F80077251209947F007E007D207C411242BE34
:10110800907702120994907702E0F8A3E0F9A3E03F
:10111800FAA3E0FBE4FFFE7D807C3F120079C00467
:10112800C005C006C007E4FFFE7D807C3F907702C3
:10113800E0F8A3E0F9A3E0FAA3E0FB12007DD003F6
:10114800D002D001D0001202779076DC1209947F89
:10115800DA7E0F7D497C40900024E0F8A3E0F9A3F3
:10116800E0FAA3E0FB12016EE4FBFA79347843124B
:10117800027712417EC004C005C006C007E4FFFE26
:10118800FD7C40907702E0F8A3E0F9A3E0FAA3E041
:10119800FB12016ED003D002D001D00012016EC044
:1011A80004C005C006C007907702E0FCA3E0FDA3D9
:1011B800E0FEA3E0FF907702E0F8A3E0F9A3E0FAED
:1011C800A3E0FB12016EE4FBFA7980783F12007D00
:1011D800D003D002D001D000120079C004C005C0ED
:1011E80006C007907702E0FCA3E0FDA3E0FEA3E0C1
:1011F800FF907702E0F8A3E0F9A3E0FAA3E0FB127E
:10120800016EA804A905AA06AB07E4FFFE7D807C51
:101218003F120079E4FBFA7948784212016ED00354
:10122800D002D001D0001202779076441209947F40
:10123800DA7E0F7D497C40900024E0F8A3E0F9A312
:10124800E0FAA3E0FB12016EE4FBFA79347843126A
:10125800027712417EC004C005C006C007E4FFFE45
:10126800FD7C40907702E0F8A3E0F9A3E0FAA3E060
:10127800FB12016ED003D002D001D00012016EC063
:1012880004C005C006C007907702E0FCA3E0FDA3F8
:10129800E0FEA3E0FF907702E0F8A3E0F9A3E0FA0C
:1012A800A3E0FB12016EE4FBFA7980783F12007D1F
:1012B800D003D002D001D000120079C004C005C00C
:1012C80006C0077FDA7E0F7D497C40900024E0F855
:1012D800A3E0F9A3E0FAA3E0FB12016EE4FBFA79BC
:1012E800347843120277124194C004C005C006C086
:1012F80007E4FFFEFD7C40907702E0F8A3E0F9A345
:10130800E0FAA3E0FB12016EA804A905AA06AB0740
:10131800D007D006D005D00412016EE4FBFA794854
:10132800784212016ED003D002D001D000120277A9
:10133800907635120994907643E070387F6612648F
:10134800DA7F3A1264DA90772474FFF0A37414F009
:10135800A374F2F090771BE0FFA3E0907727CFF01B
:10136800A3EFF07B017A76795412306C7F05126412
:09137800411247CF9076E6E0FF38
:011381002249
:10611800E6FDEDFF7851EEF6FE08EFF6FFFDAC0662
:04612800E4120386F4
:10612C0090772112099490769BE0FCA3E0FDA3E00C
:10613C00FEA3E0FF907721E0F8A3E0F9A3E0FAA337
:10614C00E0FB12016EE4FBFA7980784512027722AB
:1000260090769AE014600304701A90771FE4F0A3A8
:100036007400F0A37429F0A37410F07BFF7A1C7986
:1000460069125A2B90772474FFF0A37415F0A374E9
:1000560014F0900018E0907727F07B007A00793949
:0D00660012306C125F177F207EA102662C05
:105FB30090769AE014600304701A90771FE4F0A3BC
:105FC3007400F0A37429F0A37410F07BFF7A1C799A
:105FD3008B125A2B90772474FFF0A37415F0A374DB
:105FE30014F090000CE0907727F07B007A00793969
:0D5FF30012306C125F177F207EA102662C19
:104A5200900014E064507004A3E06431702B9076EF
:104A6200F7E024FE601204701E9076E9E024FE60F6
:104A720005047041802D80319076E9E024FE6005C6
:104A82000470598045804980599076F7E024FE6091
:104A92002A04704E9076E0E024FE600D146010242B
:104AA2000270127EFF7FF6803C7EFF7F9C80367E06
:104AB200FC7F18803074FFFEFF802A9076E0E024AD
:104AC200FE600D146010240270127E007F0A8015B1
:104AD2007E007F64800F7E037FE880097E007F0175
:104AE2008003E4FEFF908002E0FD907714E4F0A3DF
:074AF200EDF0E49076F7F00F
:014AF900229A
:10348A00900000E0FCA3A3A3E4FFFEFDEC78181271
:10349A0008B3900028EFF0900000A3E0FDA3A3E496
:1034AA00FFFEE4FC78101208B3900029EFF09000B8
:1034BA0000A3A3E0FEA3E4FFE4FDFC78081208B32E
:1034CA0090002AEFF0900000A3A3A3E0FF90002B46
:1034DA00EFF0907629E0FCA3A3A3E4FFFEFDEC78CD
:1034EA00181208B390002CEFF0907629A3E0FDA300
:1034FA00A3E4FFFEE4FC78101208B390002DEFF06D
:10350A00907629A3A3E0FEA3E4FFE4FDFC78081269
:10351A0008B390002EEFF0907629A3A3A3E0FF90C2
:10352A00002FEFF090768CE0900030F090768DE0EE
:10353A00900031F0907714E4F0A37410F09000003A
:10354A00E0FCA3E0FDA3E0FEA3E0FF124424907791
:10355A002474FFF0A37415F0A37426F09076F2E0B9
:10356A00FCA3E0FDA3E0FEA3E0FF907727120994F5
:10357A007B007A00793912306C78487620125F170E
:10358A00120A449076F2E0F8A3E0F9A3E0FAA3E085
:10359A00FB90768CE0FEA3E0FFEE3395E0FDFCEBBA
:1035AA002FFFEA3EFEE93DFDE83CFC1244249076FA
:1035BA0044E0FF907714E475F001120761FC742867
:1035CA0025F0F58274003CF583EFF0907645E0FF34
:1035DA00907714E475F001120761FC742825F0F560
:1035EA008274003CF583EFF0907646E0FF90771402
:1035FA00E475F001120761FC742825F0F582740065
:10360A003CF583EFF0907647E0FF907714E475F08D
:10361A0001120761FC742825F0F58274003CF583D9
:10362A00EFF0907635E0FF907714E475F001120719
:10363A0061FC742825F0F58274003CF583EFF09064
:10364A007636E0FF907714E475F001120761FC7496
:10365A002825F0F58274003CF583EFF0907637E088
:10366A00FF907714E475F001120761FC742825F0C5
:10367A00F58274003CF583EFF0907638E0FF90779E
:10368A0014E475F001120761FC742825F0F58274C0
:10369A00003CF583EFF09076DCE0FF907714E47558
:1036AA00F001120761FC742825F0F58274003CF5DC
:1036BA0083EFF09076DDE0FF907714E475F0011265
:1036CA000761FC742825F0F58274003CF583EFF05D
:1036DA009076DEE0FF907714E475F001120761FC42
:1036EA00742825F0F58274003CF583EFF09076DFBC
:1036FA00E0FF907714E475F001120761FC74282545
:10370A00F0F58274003CF583EFF0907702E0FF90C9
:10371A007714E475F001120761FC742825F0F5822C
:10372A0074003CF583EFF0907703E0FF907714E4A0
:10373A0075F001120761FC742825F0F58274003CCB
:10374A00F583EFF0907704E0FF907714E475F001C9
:10375A00120761FC742825F0F58274003CF583EFAA
:10376A00F0907705E0FF907714E475F00112076195
:10377A00FC742825F0F58274003CF583EFF0900084
:10378A0020E0FF907714E475F001120761FC7428B9
:10379A0025F0F58274003CF583EFF0900021E0FFFC
:1037AA00907714E475F001120761FC742825F0F58E
:1037BA008274003CF583EFF0900022E0FF907714CA
:1037CA00E475F001120761FC742825F0F582740093
:1037DA003CF583EFF0900023E0FF907714E475F056
:1037EA0001120761FC742825F0F58274003CF58308
:1037FA00EFF0900024E0FF907714E475F0011207CF
:10380A0061FC742825F0F58274003CF583EFF09092
:10381A000025E0FF907714E475F001120761FC744B
:10382A002825F0F58274003CF583EFF0900026E03D
:10383A00FF907714E475F001120761FC742825F0F3
:10384A00F58274003CF583EFF0900027E0FF907753
:10385A0014E475F001120761FC742825F0F58274EE
:10386A00003CF583EFF0907629E0FCA3E0FDA3E0AD
:10387A00FEA3E0FF9076F2E0F8A3E0F9A3E0FAA352
:10388A00E0FBD31208A250030235587E207DFF7C4C
:10389A005F1250AD90000CEFF012549D900014E0AE
:1038AA00FEA3E0FF900010EEF0A3EFF08E22F523C6
:0138BA0022EB
:02644100A907A9
:10644300E4FBFA74542BF582E43476F583E0FF120F
:1064530064DAE9FF0BEBAC0270010A14C39FEC94FE
:086463000040E07F200264DA32
:1023E00090769AE014601C04703390771FE4F0A399
:1023F0007400F0A37429F0A37420F07BFF7A1B799A
:10240000B2801790771FE4F0A37400F0A37429F052
:10241000A37420F07BFF7A1B79E4125A2B125F170A
:102420007F007E207B017A0079287DFF7C5F124C43
:102430004490000CEFF0900028E0FFE4FCFDFE78F3
:10244000181208C6900000120994900000E0F8A34A
:10245000E0F9A3E0FAA3E0FBC000900029E0FFE46C
:10246000FCFDFE78101208C6D000EB4FFFEA4EFECE
:10247000E94DFDE84CFC900000120994900000E04A
:10248000F8A3E0F9A3E0FAA3E0FBC00090002AE083
:10249000FFE4FCFDFE78081208C6D000EB4FFFEA0F
:1024A0004EFEE94DFDE84CFC9000001209949000AE
:1024B00000E0F8A3E0F9A3E0FAA3E0FB90002BE032
:1024C000FFEB4FFFEAFEE9FDE8FC900000120994E3
:1024D00090002CE0FFE4FCFDFE78181208C6907610
:1024E00029120994907629E0F8A3E0F9A3E0FAA371
:1024F000E0FBC00090002DE0FFE4FCFDFE78101230
:1025000008C6D000EB4FFFEA4EFEE94DFDE84CFC5B
:10251000907629120994907629E0F8A3E0F9A3E0D7
:10252000FAA3E0FBC00090002EE0FFE4FCFDFE7883
:10253000081208C6D000EB4FFFEA4EFEE94DFDE859
:102540004CFC907629120994907629E0F8A3E0F9E2
:10255000A3E0FAA3E0FB90002FE0FFEB4FFFEAFEC1
:10256000E9FDE8FC907629120994900030E07F00A4
:10257000FE90768CF0A3EFF0900031E0FDEDFF903F
:10258000768CEEF0A3EFF0E490771AF0A3F07FDC06
:102590007E05FDFC900000E0F8A3E0F9A3E0FAA3BB
:1025A000E0FBC31208A250129000001209A0000024
:1025B00005DC90771AE4F0A304F0E47FB87E88FD90
:1025C000FC907629E0F8A3E0F9A3E0FAA3E0FBD3BE
:1025D0001208A240149076291209A0000088B89031
:1025E000771AE0F0A3E04402F090768CE0FEA3E0DE
:1025F000FFC39401EE64809480400BD3EF94E8EE27
:1026000064809483401390768CE4F0A37432F0904D
:10261000771AE0F0A3E04404F0900002E0FFA3E0AA
:10262000907714CFF0A3EFF012661190771AE0FEC6
:10263000A3E0FF4E602890772474FFF0A37415F098
:10264000A37435F0A3EEF0A3EFF07B017A76795412
:1026500012306C7F19126441126673022A897F530B
:102660001264DA7F531264DA7F201264DA907724DE
:1026700074FFF0A37414F0A374F2F0900002E0FF72
:10268000A3E0907727CFF0A3EFF07B017A7679541F
:1026900012306C7F051264417F531264DA7F451259
:1026A00064DA7F201264DA90772474FFF0A3741444
:1026B000F0A374F2F090762BE0FFA3E0907727CFA1
:1026C000F0A3EFF07B017A76795412306C7F05121B
:1026D00064417F531264DA7F541264DA7F201264FB
:1026E000DA90772474FFF0A37414F0A374F2F090DE
:1026F000768CE0FFA3E0907727CFF0A3EFF07B018B
:102700007A76795412306C7F0512644112667390A8
:10271000768CE0FEA3E0FFC3907715E09FF0907702
:1027200014E09EF0907718E4F0A37410F0E4907732
:1027300016F0A3F0900000E0F8A3E0F9A3E0FAA3FC
:10274000E0FB907629E0FCA3E0FDA3E0FEA3E0C35C
:102750009BFFEE9AFEED99FDEC98FCC006C0079039
:10276000768CE0FEA3E0FBAA06EA3395E0F9F8D008
:1027700007D006120802D3907717E09F907716E0F3
:102780009E4003022A8990768CE0FEA3E0FF9077BA
:1027900015E02FF0907714E03EF07F661264DA7F48
:1027A0003A1264DA90772474FFF0A37414F0A374DF
:1027B000F2F0907714E0FFA3E0907727CFF0A3EF3B
:1027C000F07B017A76795412306C7F051264419067
:1027D0007718E475F001120761FE742825F0F58280
:1027E00074003EF583E0907644F0907718E475F03D
:1027F00001120761FE742825F0F58274003EF5830E
:10280000E0907645F0907718E475F001120761FECC
:10281000742825F0F58274003EF583E0907646F04A
:10282000907718E475F001120761FE742825F0F521
:102830008274003EF583E0907647F0907718E47557
:10284000F001120761FE742825F0F58274003EF550
:1028500083E0907635F0907718E475F00112076107
:10286000FE742825F0F58274003EF583E0907636FC
:10287000F0907718E475F001120761FE742825F0D6
:10288000F58274003EF583E0907637F0907718E497
:1028900075F001120761FE742825F0F58274003E80
:1028A000F583E0907638F0907635E0FCA3E0FDA368
:1028B000E0FEA3E0FFE4FBFA798078BF12016E909E
:1028C0007635120994907718E475F001120761FECD
:1028D000742825F0F58274003EF583E09076DCF0F4
:1028E000907718E475F001120761FE742825F0F561
:1028F0008274003EF583E09076DDF0907718E47501
:10290000F001120761FE742825F0F58274003EF58F
:1029100083E09076DEF0907718E475F0011207619D
:10292000FE742825F0F58274003EF583E09076DF92
:10293000F0907718E475F001120761FE742825F015
:10294000F58274003EF583E0907702F0907718E40A
:1029500075F001120761FE742825F0F58274003EBF
:10296000F583E0907703F0907718E475F001120793
:1029700061FE742825F0F58274003EF583E09077BF
:1029800004F0907718E475F001120761FE742825B1
:10299000F0F58274003EF583E0907705F0907718AB
:1029A000E475F001120761FE742825F0F5827400C9
:1029B0003EF583E0900020F0907718E475F0011266
:1029C0000761FE742825F0F58274003EF583E090DF
:1029D0000021F0907718E475F001120761FE742869
:1029E00025F0F58274003EF583E0900022F09077A8
:1029F00018E475F001120761FE742825F0F5827461
:102A0000003EF583E0900023F0907718E475F00124
:102A1000120761FE742825F0F58274003EF583E00C
:102A2000900024F0907718E475F001120761FE74AD
:102A30002825F0F58274003EF583E0900025F090A3
:102A40007718E475F001120761FE742825F0F5820D
:102A500074003EF583E0900026F0907718E475F05E
:102A600001120761FE742825F0F58274003EF5839B
:102A7000E0900027F01247CF907717E004F070063F
:102A8000907716E004F002273490772474FFF0A3C7
:102A90007414F0A374F6F07B017A76795412306CDA
:082AA0007F021264410266731B
:1047CF0090772474FFF0A37415F0A37451F09076D2
:1047DF0044E0FCA3E0FDA3E0FEA3E0FF90772712E7
:1047EF0009947B017A76795412306C7F0B126441F5
:1047FF0090772474FFF0A37415F0A3745AF0907699
:10480F0035E0FCA3E0FDA3E0FEA3E0FF90772712C5
:10481F0009947B017A76795412306C7F0B126441C4
:10482F0090772474FFF0A37415F0A37463F090765F
:10483F00DCE0FCA3E0FDA3E0FEA3E0FF90772712EE
:10484F0009947B017A76795412306C7F0C12644193
:10485F0090772474FFF0A37415F0A3746DF090009B
:10486F0020E0FCA3E0FDA3E0FEA3E0FF907727127A
:10487F0009947B017A76795412306C7F0C12644163
:10488F007F201264DA90772474FFF0A37415F0A3DD
:10489F007477F0900024E0FCA3E0FDA3E0FEA3E01A
:1048AF00FF9077271209947B017A76795412306C36
:0D48BF007F0C1264417F201264DA026673E0
:102AA800E4907643F0900018F090000C04F0123B8C
:102AB80073C298D2ACD29CE49076CBF09076A1F019
:102AC8009076E07403F0E49076E9F090001EF0A3AD
:102AD800F09076F6740FF0E4900014F0A3F090767E
:102AE8004EF090770104F0D2A8C298D2AFC2A9C222
:102AF8008CC28DE49076E5F090770B04F0A374F522
:102B0800F0752210752300124F29121CAD90001485
:102B1800E0FEA3E08EF0120A172B6510112B65104A
:102B2800212B6510312B6510412B6510512B651039
:102B3800612B6510712B6510812B6510912C42203B
:102B4800312C4220512C4830212C7630412CFB501E
:102B5800512D0060212D11607100002D2690770BFA
:102B680074FFF5F012076145F06003022D26907698
:102B7800D2120A4790770B7401F0A374F4F0900016
:102B880019E0602390770EE004F0C394025007E444
:102B980090770DF0801790770D7401F0A3E0D3942F
:102BA80003400AE4F0800690770D7401F090770DE9
:102BB800E06065900014E0FEA3E08EF0120A172B87
:102BC800E310112C0710312C0C10412C1110512C32
:102BD8001610612C1B109100002C3A124B9F907616
:102BE8004FE0FCA3E0FDA3E0FEA3E0FFEC4D4E4F59
:102BF80070407838209504764C80377620803312E0
:102C08006328802E12635A802912621D8024126262
:102C180054801F125212801A90772474FFF0A37404
:102C280014F0A374E1F07B007A00793912306C1249
:102C38005F17E4FF126573022D261238BB022D269A
:102C4800907706E475F001120761FED3E5F094E889
:102C5800EE94035003022D26123DA690772474FFAC
:102C6800F0A37415F0A37481F0907632802C9077DD
:102C780006E475F001120761FED3E5F094E8EE94DE
:102C8800035003022D26123DA690772474FFF0A36B
:102C98007415F0A37491F0907639E0FCA3E0FDE49C
:102CA80012038690769BE0F8A3E0F9A3E0FAA3E08C
:102CB800FB12016EE4FBFA7980784512027790776F
:102CC800271209947B007A00792912306C90771FBB
:102CD800E4F0A37400F0A37439F0A37410F07BFF40
:102CE8007A167947125A2B125F17E4907706F0A3E9
:102CF800F0802B12348A80261223E012557190003E
:102D0800107460F0A37431800F123F861255DB9067
:102D180000107460F0A37481F0752260F52390763A
:102D28004FE0FCA3E0FDA3E0FEA3E0FFEC4D4E4F17
:102D3800601890764F74FF120920E47B01FAF9F8C5
:102D4800C31208A27004FF1249A89076F7E0700336
:102D5800022FC9E4907710F0124A52907712EEF0E1
:102D6800A3EFF0E490770FF0900014E0FEA3E08E5C
:102D7800F0120A172E4A10112E4A10312E4A10410D
:102D88002E4A10512E4A10612E4A10912DA450112E
:102D98002DC350212DE3503100002E64900000E037
:102DA800FCA3E0FDA3E0FEA3E0FF9076E112099406
:102DB80090770F7401F0A3F0022E64907629E0FC5E
:102DC800A3E0FDA3E0FEA3E0FF9076E11209949052
:102DD800770F7402F0A314F0022E64907712E0FECD
:102DE800A3E0FF90768DE02FF090768CE03EF09097
:102DF80076D6E0FEA3E0FFC390768DE09FEE648078
:102E0800F890768CE06480985005EEF0A3EFF0D34C
:102E180090768DE0940090768CE0648094805005E4
:102E2800E4F0A304F0D390768DE094E890768CE0FB
:102E38006480948340077403F0A374E8F012595C2B
:102E4800801A9077107401F09076D2E0FCA3E0FD30
:102E5800A3E0FEA3E0FF9076E1120994907710E0DA
:102E68007003022FC99076E3E0FEA3E0FF9077138A
:102E7800E02FFF907712E03EFEF0A3EFF0E4FCFDB8
:102E88009076E1120994900014E0FEA3E08EF0120F
:102E98000A172EA650112ECD502100002F03907630
:102EA80029E0FCA3E0FDA3E0FEA3E0FF9076E1E0CB
:102EB800F8A3E0F9A3E0FAA3E0FBD31208A2403B91
:102EC8009076298025900000E0FCA3E0FDA3E0FEB9
:102ED800A3E0FF9076E1E0F8A3E0F9A3E0FAA3E02D
:102EE800FBC31208A25014900000E0FCA3E0FDA36D
:102EF800E0FEA3E0FF9076E1120994E47FDC7E0512
:102F0800FDFC9076E1E0F8A3E0F9A3E0FAA3E0FB8A
:102F1800D31208A2500A9076E11209A0000005DC3D
:102F2800E47FD07E84FDFC9076E1E0F8A3E0F9A38D
:102F3800E0FAA3E0FBC31208A2400A9076E1120966
:102F4800A0000084D0E4907711F0900014E0FEA374
:102F5800E08EF0120A172F6A50112F8950210000B5
:102F68002FA89076E1E0FCA3E0FDA3E0FEA3E0FF3C
:102F780090000012099412646B90770F7401F0802E
:102F8800389076E1E0FCA3E0FDA3E0FEA3E0FF902B
:102F9800762912099412649490770F7402F08019BC
:102FA8009076E1E0FCA3E0FDA3E0FEA3E0FF9076CD
:102FB800D2120994E490770FF090770FE0FF12494E
:102FC800A89076AE74FF120955E4FBFAF9F8C3121B
:102FD80008A27013908002E0751800F5199076AE7B
:102FE8001209A0000003E8900018E0600312002610
:0F2FF80090000CE06003022B12125FB3022B1249
:1000760002042BE86480F8E933E83360110460F089
:10008600ED33EC337009E8FCE9FDEAFEEBFF2204F0
:1000960060DED3EB9FEA9EE99DE8C2E78CF0C2F7EB
:1000A60095F0400CE8CCF8E9CDF9EACEFAEBCFFBB7
:1000B6001203F685D0F05804700320D5B3E8047017
:1000C600075002B2D502043592D5EC0460F7E4CCB1
:1000D600C0E0C398F8603B94186008400DD0E0FB80
:1000E60002040DE4FBFAC9FC8028E830E406E4C902
:1000F600FBE4CAFCE830E305E4C9CACBFCE85407D4
:100106006010F8C3E913F9EA13FAEB13FBEC13FCDE
:10011600D8F130F52FC3E49CFCEF9BFFEE9AFEED81
:1001260099FDD0E0FBEF4E4D4C701222DB0302042A
:1001360032EC2CFCEF33FFEE33FEED33FDED30E712
:10014600EB02040DEF2BFFEE3AFEED39FDD0E0FB9E
:1001560050130BBB0003020435ED13FDEE13FEEF47
:0801660013FFEC13FC02040D71
:10016E00EC4D6011E8497017ED33EC3304600DE48B
:10017E00FCFFFEFD22E933E8330470F802042B1273
:10018E0003F658046009E4CC248150062850090275
:10019E000435284003020432C0E0EB4A7044B980B3
:1001AE0006D0E0FB020421EF4E701CBD8008EBFF71
:1001BE00EAFEE9FD80EBE98DF0A4FEE5F0020257C0
:1001CE00E9CDF9EAFEEBFFEF89F0A4FCE5F0CE896C
:1001DE00F0A42EFFE435F0CD89F0A42DFEE435F029
:1001EE008067EF4E7005BD80D780C3EF8BF0A4AC57
:1001FE00F0EE8BF0A42CFCE435F0F8EF8AF0A42C92
:10020E00E5F038FCE433CB8DF0A42CFCE5F03BF8A4
:10021E00EE8AF0A42CFCE5F038F8E433CF89F0A494
:10022E002CFCE5F038CF3400CE89F0A42FFFE5F09A
:10023E003EFEE433C98DF0A42EFEE5F039CD8AF0F2
:10024E00A42FFFE5F03EFEE43DFD33D0E0FB50076A
:10025E000BBB000F020435EC2CFCEF33FFEE33FE2C
:06026E00ED33FD02040D5A
:10027400020435EC5D046005E85904700302042BA4
:100284001203F6580460F6EC4860F2EC7004FDFECC
:10029400FF22C860DB2481C85009C398600250065D
:1002A4000204329850CAF582E9294B4A7005AB82A0
:1002B40002042175F0007C1A7880C3EF9BEE9AED5E
:1002C40099400DC3EF9BFFEE9AFEED99FDE842F0D5
:1002D400DC23ACF0D0E0FFD0E0FED0E0FDAB822028
:1002E400E7101BEB60BAEC2CFCEF33FFEE33FEEDB2
:1002F40033FD02040DE803F830E705C0F075F000A3
:10030400EF2FFFEE33FEED33FD40B830E7C280AA95
:1003140074F8CC6480CCC86480C8F582046043C39C
:10032400EB9FF5F0EA9E42F0E99D42F0E89C45F02F
:1003340060305018E5825FFFE582F42B5582FB5054
:10034400210ABA001D09B90019088016E5825BFB71
:10035400E582F42F5582FF50090EBE00050DBD0045
:10036400010CC3EB9FF5F0EA9E42F0E99D42F0E8F0
:0D0374009C45F06007CC4820E701B3EC2267
:1003810075F020800E75F010800575F0087D007EF7
:10039100007F003392D530D503120894EC3340101E
:1003A100EF33FFEE33FEED33FDEC33FCD5F0ED2200
:0E03B100E5F0247EA2D513CC92E7CDCEFF223C
:1003BF00EDD2E7CD33EC3392D524814006E4FFFE36
:1003CF00FDFC22FCE4CFCECDCC24E0501174FF8095
:1003DF00EDC3CC13CCCD13CDCE13CECF13CF047032
:0703EF00F030D5DE02089496
:10300700E51A2424F582E43477F583E0051A229043
:103017007721300703907724E475F0011209D10274
:10302700066A2000E97F2ED2008018EF540F249003
:10303700D43440D4FF30040BEF24BFB41A0050033C
:103047002461FFE51B6002151B051EE51E700205C6
:103057001D30070E907721E475F0011209D1EF02B8
:1030670006B00264E47403D2078003E4C207F51ACA
:103077009077211209E8E4F51BF51DF51EE51B60A5
:10308700077F2012304A80F5751CFFC201C200C2BB
:1030970002C203C205C206C208123016FF700D3005
:1030A70007057F0012305BAF1EAE1D22B4255FC23D
:1030B700D5C204123016FF24D0B40A00501A75F096
:1030C7000A781B30D50508B6FF0106C6A426F620E8
:1030D700D5047002D20380D924CFB41A00EF50046C
:1030E700C2E5D20402334DD20180C6D20080C0D2DD
:1030F7000280BCD2D580BAD20580B47F2012304A74
:103107002002077401B51B0040F1123007FF12308F
:103117004A023084D208D2068095123007FB12305B
:1031270007FA123007F94A4B7006794B7A347BFF5E
:1031370020022EE51B602A7E008E82758300120610
:103147008360060EEE651C70F0C2D5EBC0E0EAC0E6
:10315700E0E9C0E0EE1233AED0E0F9D0E0FAD0E01B
:10316700FB12066AFF60AAEBC0E0EAC0E0E9C0E034
:1031770012304AD0E02401F9D0E03400FAD0E0FB65
:10318700E51C0460DCD51CD98087D20280A21233EB
:103197009060F7E51C70010412046BA91C600DE533
:1031A7001C600914F51C123438EF60F3EA30E702AB
:1031B700F404C3995079EAF4251C0430E701E404C8
:1031C700F51C800D12339060C1EA051C251C120402
:1031D7006BEA907750F030E701E4251C04D51C0416
:1031E700200501141233AEE4C0E012343890775052
:1031F700E0601320E70714F0123032802204F0D089
:10320700E014C0E07F00123032E51C60071230295D
:10321700151C800B300503123029D0E0023084D012
:10322700E00480C4123390609EE51C0412046B9086
:103237007750EAF0E51C20050260010424041233EC
:01324700AED8
:1032480074FF04C0E0123438123032E51C20050245
:103258006003123029D0E0B51CE87F4512303C905D
:103268007750E07F2B30E7047F2DF404C0E0123064
:103278004AD0E075F00A84C0F0123033D0E0123042
:1032880033023084791080027908C206C2088008A7
:10329800D2D5790A8004790AC2D5E51C047002F5F2
:1032A8001CE4FAFDFEFF123007FC7B082001131214
:1032B8003007FD7B1030000A123007FE123007FF7E
:1032C8007B20EC3382D592D55013C3E43000069F9F
:1032D800FFE49EFEE42001039DFDE49CFCE4CBF8A2
:1032E800C201EC700CCFCECDCCE824F8F870F38096
:1032F80017C3EF33FFEE33FEED33FDEC33FCEB3356
:10330800FB994002FB0FD8E9EB300105F8D0E0C487
:1033180048B201C0E00AEC4D4E4F78207B0070C2E5
:10332800EAB51C0040BCC0E01233B0D0F0D0E020B9
:103338000104C4C0E0C4B201C0F0123033D0F0D5EB
:10334800F0EB0230841209F1312153328C5830F2FB
:103358004C30EE4232904F3298443298493107430C
:10336800329E5531CB46322B45319547346B503020
:10337800F62D30FA2E311D2B30FE23311B2034540C
:103388002A30B64800003115E51CB4FF03751C0649
:10339800123007FC123007FD123007FE123007FF0B
:1033A8009077490204A8790AA2D5200314300509A8
:1033B800B910020404B9080104A2D520060250017C
:1033C800042002689202B51B005034C0E07F203010
:1033D80003197F30A20272067205500F123407C219
:1033E80002C206C205C2087F30800F300503E9C05B
:1033F800E012304A300503D0E0F9D0E0B51BCC30FC
:1034080005177F30B9100C12304A7F583004077FF7
:10341800788003B9080312304A3002057F2D023044
:103428004A7F202008F87F2B2006F322920280CFC3
:103438007F00B40700500B2449F582E43477F58304
:10344800E0FF22286E756C6C2900D201123007301B
:1034580001F8C201781B30D50108F60230B62D50AC
:103468004349581230072403B405004001E490345E
:10347800669312303B743A12303BD203751B040238
:02348800328C84
:104136003A70FA83BCAAE9E43E81E0F8BF9DE9E65D
:104146003F80000039283C1ABB9969663DA335E3D8
:10415600BF255DE73FC90FDB418DDBCCC44936EE99
:1041660045C9913FC5B0F83D3F800000C317F534FF
:10417600452FFA73C60AFDDD12423F04A2E1920002
:104186001420E01590413674041205AD80301242B9
:104196003F30E102B20020E0EBA883A982907721AC
:1041A6001209948982888390414A74041205AD8568
:1041B60082F090772112090285F08212016EED4C91
:1041C6006007300004EC6480FC2212423FC0E0A885
:1041D60083A9829077211209948982888390416EFF
:1041E60074031205AD8582F090772112090285F0DD
:1041F6008212016E907721E0CCF0A3E0CDF0A3E02F
:10420600CEF0A3E0CFF090415E74031205ADD082EC
:104216008582F090772112090285F082E58230E0EE
:1042260007120277B2008096EFCBFFEECAFEEDC909
:10423600FDECC8FC1202778085ED33EC547FCC335D
:10424600920024605007D0E0D0E002042B7B837AF2
:10425600F97922783E12016EEDF933ECF8332481B8
:104266005011EFFBEEFA1203BF120381ECB2E7FC2A
:1042760012007DED33EC33602F2403F8C313FCEDFD
:1042860092E7FDE82481E4501FECF8EDF9EEFAEF31
:10429600FB1203BFEF04C2E0FCF58212038BECB203
:1042A600E7FC12007DE58203FAED33EC3360071478
:0842B60013FCED92E7FDEA2282
:1042BE00907721120994E4FFFE7D807C3F90772158
:1042CE00E0F8A3E0F9A3E0FAA3E0FB1203147006F2
:1042DE00907721024418907721E0FCA3E0FDA3E043
:1042EE00FEA3E0FF120440FBA3E0FCA3E0FDA3E06D
:1042FE00FEA3E0FF120440FFB40108E4FFFE7D8040
:10430E007C3F22EF64046029EB64046024EBB4016B
:10431E0030E4FFFEFDFC907725E0F8A3E0F9A3E082
:10432E00FAA3E0FB12031460084006E4FFFEFDFC56
:10433E00229077251209A0FFFFFFFF9077250244F8
:10434E0018E4907729F0A3F0FFFEFDFC907721E0B2
:10435E00F8A3E0F9A3E0FAA3E0FB120314505F9078
:10436E007725E0FCA3E0FDA3E0FEA3E0FF1203BF70
:10437E00907729EEF0A3EFF0FDCCEECCEC12038695
:10438E00C8ECC8C9EDC9CAEECACBEFCB907725E011
:10439E00FCA3E0FDA3E0FEA3E0FF120079E4FBFA2C
:1043AE00F9F8120314708A907721E0FCA3E0FDA3C4
:1043BE00E0FEA3E0FF12045A907721120994907741
:1043CE0021E0FCA3E0FDA3E0FEA3E0FF1246DA909D
:1043DE007725E0F8A3E0F9A3E0FAA3E0FB12016E63
:1043EE00124D1D90772512099490772AE030E01730
:1043FE00907725E0FCA3E0FDA3E0FEA3E0FF12040E
:10440E005A907725120994907725E0FCA3E0FDA33E
:06441E00E0FEA3E0FF2216
:1003F600E9D2E7C933E833F892D5EDD2E7CD33EC4D
:0704060033FC5002B2D522C5
:10040D00EC30E7100FBF000C0EBE00080DBD000450
:10041D000BEB6014A2D5EB13FCED92E7FD2274FFFC
:10042D00FCFDFEFF22E480F8A2D574FF13FC7D8055
:03043D00E480EF69
:10044000ED33EC33601004700FED547F70057402CF
:0A04500092E2227404220422E42246
:10045A00ED33EC33600A047003BD8004ECB2E7FCB0
:01046A00226F
:10046B00F920E73624F950037907E4F42402FBE57D
:10047B0082158270021583DBF6E024FB501BE960CA
:10048B0014E4F0E582158270021583E004F0B40ADF
:0D049B0008E4F0D9EE7401F00A22C2D52267
:1004A800ED33EC3392D5FA602AB4FF33EDC2E77B23
:1004B800FF60067A0479CDE4227A0479D620D5043F
:1004C8007A0479D1224E614E002B494E46002D49BF
:1004D8004E4600E47A08F0A3DAFC7B00740722C0D9
:1004E80083C082ECC0E0EDC0E0EEC0E0EFC0E0EA1F
:1004F80075F010A4CAABF075F04DA42BFBE435F0F1
:10050800FCEA2410FAEB34C5FBEC34D9FCEDC2E765
:10051800FF75F056A4F42411C5F0F434C58FF0A487
:100528002AE5F03BE43CF020E71412062AD0E0FF6D
:10053800D0E0FED0E0FDD0E0FC1202778014F40495
:1005480012062AD0E0FFD0E0FED0E0FDD0E0FC1299
:10055800016ED082D083E0FAEDD2E7CD33EC3324BC
:1005680082FBE4C3CF33CFCE33CECD33CD33DBF3F1
:100578007B0775F00A846004F0A31B0AE5F0F0A37A
:100588008FF0740AA4FFACF08EF0740AA42CFEACB1
:10059800F050010C8DF0740AA42CFDE435F0F0A3A2
:0505A800DBDE740722F8
:1005AD00C0E0EFFBEEFAEDF9ECF812016ED0E0F5DC
:1005BD00F0EFFBEEFAEDF9ECF81208E5A3A3A3A317
:1005CD00E8C0E0E9C0E0EAC0E0EBC0E0C0F0120135
:1005DD006E12090EA3A3A3A312007DD0F0D0E0FBF1
:0D05ED00D0E0FAD0E0F9D0E0F8D5F0D4224B
:104CE50033DA929E35B16011377FE5FE392184892B
:104CF5003AAEC3FF3C1D955B3D6358473E75FDF0DD
:104D05003F3172183F800000C2D502043502042BE2
:104D1500BD80FA50F3020432ED33EC330460F17BCD
:104D25003B7AAA79B8783F12016EED33EC3392D510
:104D3500247B5011A2D570DB500BED448024045028
:104D450004A2D580CEEFFBEEFAEDF9ECF81203BF25
:104D5500EFF582F404FC12038B12007DC082904CA7
:104D6500E574091205BCED33CC33D0F092D525F0AE
:0A4D7500A2D57001C313CC13FD2278
:1046A6003E9248DA3ECCCCCD3F2AAAAB4000000071
:1046B6003F8000003F9837F03FB504F33FD744FCF6
:1046C6003E3172173EB172173F0515913EDE5BD93A
:1046D600D2008002C200EDD2E7F8CD33EC3304708D
:1046E6000BBD800592D502043502042B40FBD31482
:1046F60060F2F5F07C3FEE7A00C39496C8948B4046
:10470600230AC89469C8941A401A0AC89468C894B7
:104716001F40110AC8945AC89425400805F07A002B
:10472600CDC2E7CDC0F090772B120994EA2323C0BF
:10473600E024B6F582E43446F58312090E12007DB4
:10474600ECC0E0EDC0E0EEC0E0EFC0E01208E5909E
:10475600772B120902120079D0E0FBD0E0FAD0E004
:10476600F9D0E0B2E7F812027790772B120994900D
:1047760046A674031205AD90772B12090212016E3C
:10478600D0E0600F24C2F582E43446F58312090EA8
:1047960012007D90772B120994D0E0C3947FFDE43C
:1047A6009400FC1203867B187A727931783F1201E5
:1047B6006E90772B12090212007D30000B7BD97A9E
:0947C6005B79DE783E12016E22DF
:1005FA003F8000004120000042C80000447A000009
:10060A00461C400047C35000497424004B1896808A
:10061A004CBEBC205A0E1BCA6753C21C749DC5AE81
:10062A00FB60065407601C2323120658EB543860FB
:10063A000912064412065312016EECF8EDF9EEFAAD
:10064A00EFCB22EB12065380F1543803241C900599
:10065A00FAFE93FC0EEE93FD0EEE930ECE93FF225E
:03000000024E1499
:0C4E1400787FE4F6D8FD758188024E5BC3
:10066A00BB010689828A83E0225002E722BBFE028E
:09067A00E32289828A83E49322C1
:10068300BB010CE58229F582E5833AF583E022502C
:1006930006E92582F8E622BBFE06E92582F8E22276
:0D06A300E58229F582E5833AF583E4932290
:1006B000BB010689828A83F0225002F722BBFE0129
:0206C000F32223
:1006C200F8BB010DE58229F582E5833AF583E8F06E
:1006D200225006E92582C8F622BBFE05E92582C81A
:0206E200F22202
:1006E400EF8DF0A4A8F0CF8CF0A428CE8DF0A42E2A
:0206F400FE22E4
:1006F600BC000BBE0029EF8DF084FFADF022E4CCE8
:10070600F875F008EF2FFFEE33FEEC33FCEE9DECB0
:10071600984005FCEE9DFE0FD5F0E9E4CEFD22EDF6
:10072600F8F5F0EE8420D21CFEADF075F008EF2F40
:10073600FFED33FD4007985006D5F0F222C398FD31
:050746000FD5F0EA22CE
:10074B00C5F0F8A3E028F0C5F0F8E5821582700239
:06075B001583E038F022D6
:10076100A3F8E0C5F025F0F0E5821582700215834B
:06077100E0C838F0E822A8
:10077700E88FF0A4CC8BF0A42CFCE98EF0A42CFC21
:100787008AF0EDA42CFCEA8EF0A4CDA8F08BF0A49F
:100797002DCC3825F0FDE98FF0A42CCD35F0FCEBFE
:1007A7008EF0A4FEA9F0EB8FF0A4CFC5F02ECD39C3
:0F07B700FEE43CFCEAA42DCE35F0FDE43CFC2230
:1007C60075F008758200EF2FFFEE33FECD33CDCCEA
:1007D60033CCC58233C5829BED9AEC99E58298406D
:1007E6000CF582EE9BFEED9AFDEC99FC0FD5F0D64A
:1007F600E4CEFBE4CDFAE4CCF9A88222B800C1B974
:100806000059BA002DEC8BF084CFCECDFCE5F0CBB1
:10081600F97818EF2FFFEE33FEED33FDEC33FCEBEA
:1008260033FB10D703994004EB99FB0FD8E5E4F9A5
:10083600FA227818EF2FFFEE33FEED33FDEC33FC92
:10084600C933C910D7059BE99A4007EC9BFCE99A86
:10085600F90FD8E0E4C9FAE4CCFB2275F010EF2FCB
:10086600FFEE33FEED33FDCC33CCC833C810D707CB
:100876009BEC9AE899400AED9BFDEC9AFCE899F806
:0E0886000FD5F0DAE4CDFBE4CCFAE4C8F92299
:0E089400C3E49FFFE49EFEE49DFDE49CFC2275
:1008A200EB9FF5F0EA9E42F0E99D42F0E89C45F0AC
:0108B2002223
:1008B300E8600FECC313FCED13FDEE13FEEF13FF23
:0308C300D8F12247
:1008C600E8600FEFC333FFEE33FEED33FDEC33FC90
:0308D600D8F12234
:0C08D900E6FC08E6FD08E6FE08E6FF224B
:1008E500E493FC740193FD740293FE740393FF2259
:0D08F500E6FB08E6F908E6FA08E6CBF82273
:0C090200E0F8A3E0F9A3E0FAA3E0FB2278
:10090E00E493F8740193F9740293FA740393FB223F
:10091E007401FF3395E0FEFDFCA3A3A3E0CF2FF0FF
:10092E00E582158270021583E0CE3EF0E5821582D7
:10093E0070021583E0CD3DF0E582158270021583BD
:05094E00E0CC3CF022AA
:100953007401FF3395E0FEFDFCA3A3A3E02FFFF09A
:10096300E582158270021583E03EFEF0E582158272
:1009730070021583E03DFDF0E58215827002158358
:05098300E03CFCF02245
:0C098800ECF608EDF608EEF608EFF6229B
:0C099400ECF0A3EDF0A3EEF0A3EFF022D6
:1009A000A8828583F0D083D0821209B71209B712CA
:1009B00009B71209B7E473E493A3C583C5F0C583EF
:1009C000C8C582C8F0A3C583C5F0C583C8C582C8A1
:0109D0002204
:1009D100F8E0FBA3A3E0F925F0F0E58215827002AF
:0709E1001583E0FA38F02253
:0909E800EBF0A3EAF0A3E9F02210
:1009F100D083D082F8E4937012740193700DA3A395
:100A010093F8740193F5828883E4737402936860A8
:060A1100EFA3A3A380DFA8
:100A1700D083D082F8E4937012740193700DA3A36E
:100A270093F8740193F5828883E473740293B5F0A5
:0D0A3700067403936860E9A3A3A3A380D80D
:1064E400EFB40A07740D1264EF740A309811A89976
:1064F400B8130CC2983098FDA899C298B811F63018
:0765040099FDC299F59922EF
:104E2000022AA8E493A3F8E493A34003F68001F2D6
:104E300008DFF48029E493A3F85407240CC8C33393
:104E4000C4540F4420C8834004F456800146F6DF62
:104E5000E4800B01020408102040809060D3E47EBF
:104E6000019360BCA3FF543F30E509541FFEE49357
:104E7000A360010ECF54C025E060A840B8E493A31E
:104E8000FAE493A3F8E493A3C8C582C8CAC583CA49
:104E9000F0A3C8C582C8CAC583CADFE9DEE780BE01
:016117000087
:00000001FF
